:0200000480007A
:10000000B72F0000938F0F8073900F306F00400365
:100010001300000013000000130000001300000094
:100020001300000013000000130000001300000084
:100030001300000013000000130000001300000074
:100040009702000093824211739052309300000097
:10005000130100009301000013020000930200004E
:100060001303000093030000130400009304000036
:10007000130500009305000013060000930600001E
:100080001307000093070000130800009308000006
:100090001309000093090000130A0000930A0000EE
:1000A000130B0000930B0000130C0000930C0000D6
:1000B000130D0000930D0000130E0000930E0000BE
:1000C000130F0000930F000097110200938141D29B
:1000D0001705020013050553979503009385C57313
:1000E00013060000EF00001A17050200130505446F
:1000F000970502009385854F13060000EF008018D6
:1001000017A503001305857197B503009385C57086
:1001100037B6ABAB1306B6BAEF00C01617B1030083
:100120001301C16FEF80D0559392120093D2120049
:100130009382D2FF638A02008322010013014100EF
:100140006F0000177300203083220100130141006B
:10015000730020301301C1FF23205100F32220340B
:10016000E3C402FC8322010013014100130141F8A2
:1001700023221100232421002326310023284100BB
:10018000232A5100232C6100232E71002320810299
:10019000232291022324A1022326B1022328C10293
:1001A000232AD102232CE102232EF1022320010570
:1001B0002322110523242105232631052328410567
:1001C000232A5105232C6105232E71052320810745
:1001D000232291072324A1072326B1072328C1073F
:1001E000232AD107232CE107232EF107732520347E
:1001F000F3251034130601006F000000731015344E
:1002000083204100032181008321C10003220101D9
:1002100083224101032381018323C10103240102BD
:1002200083244102032581028325C10203260103A1
:1002300083264103032781038327C1030328010485
:1002400083284104032981048329C104032A010569
:10025000832A4105032B8105832BC105032C01064D
:10026000832C4106032D8106832DC106032E010731
:10027000832E4107032F8107832FC1071301C10775
:10028000730020302320C5006376B50013054500B8
:100290006FF05FFF678000000000000000000000BA
:1002A000000000000000000000000000000000004E
:1002B000130101F8232011002322210023243100FF
:1002C0002326410023285100232A6100232C71009A
:1002D000232E8100232091022322A1022324B10294
:1002E0002326C1022328D102232AE102232CF10272
:1002F000232E010323201105232221052324310568
:100300002326410523285105232A6105232C710545
:10031000232E8105232091072322A1072324B1073F
:100320002326C1072328D107232AE107232CF1071D
:100330009702020083A2C22223A02200F3221034DB
:10034000232E5106EF00C03B17010200032141217B
:10035000032101008322C10773901234B7220000E9
:100360009382028873A00230832001000322C1001F
:100370008322010103234101832381010324C1015D
:100380008324010203254102832581020326C10241
:100390008326010303274103832781030328C10325
:1003A000832801040329410483298104032AC10409
:1003B000832A0105032B4105832B8105032CC105ED
:1003C000832C0106032D4106832D8106032EC106D1
:1003D000832E0107032F4107832F81071301010893
:1003E00073002030970202009382C22123A01200E2
:1003F00023A2220023A4320023A6420023A85200F5
:1004000023AA620023AC720023AE820023A09202D2
:1004100023A2A20223A4B20223A6C20223A8D202CC
:1004200023AAE20223ACF20223AE020323A01205A8
:1004300023A2220523A4320523A6420523A85205A0
:1004400023AA620523AC720523AE820523A092077E
:1004500023A2A20723A4B20723A6C20723A8D20778
:1004600023AAE20723ACF207EF60903117010200E4
:100470000321010F032101008322C107739012346D
:10048000B72200009382028873A00230832001000B
:100490000322C1008322010103234101832381013F
:1004A0000324C10183240102032541028325810223
:1004B0000326C10283260103032741038327810307
:1004C0000328C103832801040329410483298104EB
:1004D000032AC104832A0105032B4105832B8105CF
:1004E000032CC105832C0106032D4106832D8106B3
:1004F000032EC106832E0107032F4107832F810797
:100500001301010873002030970202009382820FCA
:1005100083A0020003A1420083A1820003A2C200C3
:1005200083A2020103A3420183A3820103A4C201A7
:1005300083A4020203A5420283A5820203A6C2028B
:1005400083A6020303A7420383A7820303A8C2036F
:1005500083A8020403A9420483A9820403AAC20453
:1005600083AA020503AB420583AB820503ACC20537
:1005700083AC020603AD420683AD820603AEC2061B
:1005800083AE020703AFC20983AF82076780000012
:1005900073700430130101F823201100232221007D
:1005A000232431002326410023285100232A6100FF
:1005B000232C7100232E8100232091022322A102EB
:1005C0002324B1022326C1022328D102232AE102D7
:1005D000232CF102232E01032320110523222105C0
:1005E000232431052326410523285105232A6105AB
:1005F000232C7105232E8105232091072322A10797
:100600002324B1072326C1072328D107232AE10782
:10061000232CF1079702020083A282F423A0220078
:10062000232E1106EF30003317010200032141F39E
:10063000032101008322C10773901234B722000006
:100640009382028873A00230832001000322C1003C
:100650008322010103234101832381010324C1017A
:100660008324010203254102832581020326C1025E
:100670008326010303274103832781030328C10342
:10068000832801040329410483298104032AC10426
:10069000832A0105032B4105832B8105032CC1050A
:1006A000832C0106032D4106832D8106032EC106EE
:1006B000832E0107032F4107832F810713010108B0
:1006C00073002030737004306F00000073104530E9
:1006D000678000007325403073F04330678000006E
:1006E00097070000938747FE232EB5FE2322C5FA05
:1006F000232635F82320F5F8130505F86780000058
:10070000130101FF23261100EF605004EF20805CED
:10071000631805008320C1001301010167800000F8
:100720008320C100130101016F30C02293078500AF
:100730001307F0FF2322F5002324E5002326F5000C
:100740002328F500232005006780000023280500EA
:10075000678000008327450023A2F50003A78700D8
:1007600023A4E50003A787002322B70023A4B70032
:1007700023A8A50083270500938717002320F500F1
:100780006780000003A605009307F0FF13078500AC
:100790006316F6006F008003138707008327470066
:1007A00083A60700E37AD6FE23A2F50023A4B700B0
:1007B00023A4E5002322B70023A8A5008327050072
:1007C000938717002320F5006780000003270501A9
:1007D000832747006FF05FFD0327450083268500D0
:1007E000832705012324D70003278500832645009E
:1007F0002322D70003A747006316A700032785001D
:1008000023A2E7002328050003A507001305F5FF31
:1008100023A0A70067800000032605049387050036
:10082000630406028325C50003274500B385C50080
:100830002326B50063E6E500832505002326B500E1
:10084000138507006F50C04C67800000130101FF43
:100850002324810023261100130405002322910084
:10086000EF30904283278404635AF00483274402C4
:1008700063860704930444026F0000028327840404
:100880009387F7FF2324F404832784046358F0023A
:10089000832744026384070213850400EF30C06D90
:1008A000E30E05FCEF30901A832784049387F7FF4B
:1008B0002324F40483278404E34CF0FC9307F0FF23
:1008C0002324F404EF30903FEF30103C832744049E
:1008D000635AF00483270401638607049304040128
:1008E0006F000002832744049387F7FF2322F40458
:1008F000832744046358F0028327040163840702BA
:1009000013850400EF304067E30E05FCEF30101450
:10091000832744049387F7FF2322F40483274404A6
:10092000E34CF0FC9307F0FF2322F404032481003E
:100930008320C10083244100130101016F3010386E
:1009400063000508130101FF232481002322910085
:10095000130405002326110093840500EF30D032E4
:10096000832604048327C40303270400232C0402E2
:10097000B387F6021306F0FF2322C4042324E40005
:100980002324C404B386D740B307F7003307D70046
:100990002322F4002326E400639804028327040141
:1009A000639E0702EF3090318320C1000324810051
:1009B000832441001305100013010101678000002A
:1009C000737004306F00000013050401EFF01FD6B0
:1009D00013054402EFF09FD56FF0DFFC130504010F
:1009E000EF30805993071000E31EF5FAEFF05FBA7D
:1009F0006FF05FFB63160500737004306F0000003A
:100A0000130101FE232A910023282101232631010D
:100A1000232E1100232C8100930906001389050061
:100A200093040500638E05083305B50213055505CB
:100A3000EF50800D13040500630C0508930745056E
:100A40002320F500232E940223202405EF30D02309
:100A5000832604048327C403032704001306F0FF3E
:100A6000B387F602232C04022322C4042324E400C7
:100A70002324C40413050401B386D740B307F70049
:100A80003307D7002322F4002326E400EFF01FCA27
:100A900013054402EFF09FC9EF30502223083405BC
:100AA000130504008320C101032481018324410133
:100AB000032901018329C10013010102678000009D
:100AC00013054005EF5040041304050063160500AC
:100AD000737004306F000000232084006FF09FF6D5
:100AE00063160500737004306F0000006376B50074
:100AF000737004306F000000130101FF2324810094
:100B0000130620001384050093050000232611001E
:100B1000EFF05FEE630C0500232C85028320C100FB
:100B20000324810013010101678000007370043009
:100B30006F000000130101FB23261104232481040C
:100B40002322910423202105232E3103232C41034A
:100B5000232A510323286103232671032326C1007E
:100B600063060528638C052693072000639CF60026
:100B70000327C503930710006306F7007370043062
:100B80006F0000001389060093840500130405001C
:100B9000EF30C06F631A05008327C100638607002A
:100BA000737004306F000000EF30100E03278403D1
:100BB0008327C403130B0000930B20009309F0FF5D
:100BC000130A0401930A44026364F710630479234F
:100BD0008327C1006382073663160B00130581016A
:100BE000EF304054EF30900DEF20C000EF30D009CF
:100BF0008327440463943701232204048327840455
:100C00006394370123240404EF30500B9305C10093
:100C100013058101EF30005463160530EF30D00624
:100C2000032784038327C4036304F710EF301009FC
:100C3000EF309005832784046346F0026F000003C1
:100C400013850A00EF30403363040500EF30006085
:100C5000832784049387F7FF2324F40483278404E1
:100C60006356F00083274402E39C07FC23243405E9
:100C7000EF30D004EF305001832744046346F00284
:100C80006F00000313050A00EF30002F6304050016
:100C9000EF30C05B832744049387F7FF2322F404DB
:100CA000832744046356F00083270401E39C07FC78
:100CB00023223405EF309000EF204027130B100063
:100CC000EF30807C032784038327C403E370F7F0AD
:100CD0000326040463040612631A091E0325840014
:100CE00093850400EF50C002832784008326040408
:100CF00003274400B387D7002324F40063E4E710FC
:100D00008327840383260400032744029387170064
:100D10002324D400232CF40263000710130544029B
:100D2000EF308025930710006318F50E6F00401414
:100D3000EF30C0788325C10013050A00EF20D0767C
:100D4000EF308074832784046346F0026F00000351
:100D500013850A00EF30402263040500EF30004F96
:100D6000832784049387F7FF2324F40483278404D0
:100D70006356F00083274402E39C07FC23243405D8
:100D8000EF30C073EF304070832744046346F002B5
:100D90006F00000313050A00EF30001E6304050016
:100DA000EF30C04A832744049387F7FF2322F404DB
:100DB000832744046356F00083270401E39C07FC67
:100DC00023223405EF30806FEF204016E31805EE44
:100DD000EFF00FFC130B10006FF09FEE832705045C
:100DE000E38407D8737004306F0000007370043020
:100DF0006F00000003260404631006088327040024
:100E0000638607048327840303274402938717001C
:100E1000232CF402E31407F0EF30406A13051000AE
:100E20008320C10403248104832441040329010491
:100E30008329C103032A8103832A4103032B01036E
:100E4000832BC102130101056780000003254400C4
:100E5000EF308056832784030327440223220400B3
:100E600093871700232CF402E31A07EAE30605FA36
:100E7000EFF00FF26FF05FFA0325C40093850400D2
:100E8000EF401069832704040327C400832604006D
:100E9000B307F0403307F7002326E400637ED7044E
:100EA00003274400B307F7002326F40013072000AC
:100EB000832744026304E90403278403130717000C
:100EC000232CE402E38A07F46FF05FE50325C400F6
:100ED00093850400EF40D063832704040327C400F4
:100EE00083260400B307F0403307F7002326E4000D
:100EF000E37ED7FA6FF0DFFA8327440203278403E7
:100F0000E30C07FA032784031307F7FF232CE402FB
:100F10000327840313071700232CE402E38E07EE54
:100F20006FF0DFDF13050400EFF05F92EF200000A9
:100F3000130500006FF0DFEEEF304058130500009E
:100F40006FF01FEE130101FF2322910093040500AF
:100F5000130540052324810023261100EF40D03AD9
:100F600013040500630C0504232C05029307F0FF0E
:100F70002322F5041307100013050501232EE402B4
:100F80002324F40423220400232004002324040047
:100F9000232604002320040423089404EFF00FF90F
:100FA00013054402EFF08FF89306000013060000CB
:100FB0009305000013050400EFF0DFB713050400EC
:100FC0008320C10003248100832441001301010117
:100FD0006780000063040504130101FF23248100DE
:100FE00023229100232611002320210103294500FB
:100FF00013040500EF308028930400006304A90265
:101000008320C1000324810013850400032901000B
:1010100083244100130101016780000073700430D4
:101020006F0000008327C400930410009387F7FF2C
:101030002326F400E39607FC930600001306000045
:101040009305000013050400EFF0DFAE6FF05FFBC7
:101050006302050A63880508130101FE232C810041
:10106000232A91002328210123244101232E11004A
:1010700023263101930720009384060013090600FC
:10108000138A050013040500639CF6000327C503BB
:10109000930710006302F70A737004306F000000BA
:1010A000EFF04FE3032784038327C403930905006C
:1010B0006366F7049304000013850900EFF00FE165
:1010C0008320C10103248101138504000329010148
:1010D000832441018329C100032A810013010102F5
:1010E0006780000083270504E38807F673700430E7
:1010F0006F000000737004306F00000003260404CA
:10110000631E060C8327040063860712832784036B
:101110001307F0FF93871700232CF402832784041E
:101120006388E70E832784049304100093871700D5
:101130002324F4046FF05FF8EFF0CFD90327840382
:101140008327C403930905006360F706032604049C
:10115000E30A06FA0325C40093050A00EF40503B5A
:10116000832704040327C40083260400B307F04048
:101170003307F7002326E4006378D70003274400F1
:10118000B307F7002326F40093072000E390F4F858
:1011900083278403E38C07F6832784039387F7FF71
:1011A000232CF4026FF09FF603260404E30C06F4EC
:1011B0000325C40093050A00EF40903583270404FB
:1011C0000327C40083260400B307F0403307F70069
:1011D0002326E400E364D7FA6FF09FFBE39C04F658
:1011E0000325840093050A00EF4090328327840092
:1011F0008326040403274400B387D7002324F40084
:10120000E3E6E7F0832704002324F4006FF01FF0E7
:101210008327440293041000E38007EA1305440285
:10122000EF209055E30A05E8E30809E82320990038
:101230006FF09FE803254400EF30001823220400DC
:101240006FF0DFEC6302050A83270504638607005D
:10125000737004306F00000083270500638A07085D
:10126000130101FE232C8100232A910013040500A1
:101270002328210123263101232E11001389050083
:10128000EFF04FC5032784038327C40393090500A8
:10129000930400006376F702832784031307F0FFAB
:1012A00093871700232CF40283278404638AE704BE
:1012B0008327840493041000938717002324F404E5
:1012C00013850900EFF08FC08320C1010324810141
:1012D0001385040003290101832441018329C100EE
:1012E0001301010267800000737004306F0000007A
:1012F00083274500E38607F6737004306F00000013
:101300008327440263960700930410006FF05FFB8D
:1013100013054402EF205046E30805FEE30609FEEC
:10132000930710002320F9006FF01FFE130101FC4A
:10133000232E1102232C8102232A91022328210328
:101340002326310323244103232251032326C100F2
:1013500063060528638C0526938A06009389050099
:1013600013040500EF209072631A05008327C10063
:1013700063860700737004306F000000EF30C01008
:10138000832784036394071C8327C10063800710AD
:1013900013058101EF2010599304F0FF1309440253
:1013A000130A0401EF308011EF10D004EF30C00DAC
:1013B000832744046394970023220404832784042E
:1013C0006394970023240404EF30400F9305C10079
:1013D00013058101EF20105863100524EF30C00A77
:1013E00083278403638A070AEF30400DEF30C0097A
:1013F000832784046346F0026F000003130509008D
:10140000EF20903763040500EF20506483278404A5
:101410009387F7FF2324F404832784046356F000A2
:1014200083274402E39C07FC23249404EF30000943
:10143000EF308005832744046346F0026F00000309
:1014400013050A00EF20503363040500EF201060FD
:10145000832744049387F7FF2322F404832744045B
:101460006356F00083270401E39C07FC23229404C5
:10147000EF30C004EF10902BEF300001832784037E
:101480006396070C8327C100E39E07F0EF3000034B
:10149000130500006F00800FEF3040028327040027
:1014A000638807108325C10013050900EF20C07F62
:1014B000EF20907D832784046346F0026F000003D1
:1014C00013050900EF20502B63040500EF2010588E
:1014D000832784049387F7FF2324F4048327840459
:1014E0006356F00083274402E39C07FC2324940402
:1014F000EF20D07CEF205079832744046346F0022C
:101500006F00000313050A00EF2010276304050095
:10151000EF20D053832744049387F7FF2322F4045A
:10152000832744046356F00083270401E39C07FCEF
:1015300023229404EF209078EF10501F63040508D5
:10154000EF20907483278403E38E07F293850900CC
:10155000130504008324C400EFF00FAC63940A0861
:1015600083278403032704009387F7FF232CF402C7
:1015700063160700EF20D07B2322A40083270401F9
:1015800063920708EF209073130510008320C103B6
:101590000324810383244103032901038329C10216
:1015A000032A8102832A410213010104678000009B
:1015B000EF20906D03254400EF201050EF201070B5
:1015C0006FF05FEEEFE0DFFC6FF09FF7832705041D
:1015D000E38407D8737004306F0000007370043028
:1015E0006F0000008327440223269400E38C07F851
:1015F00013054402EF205018E30605F8EFE05FF909
:101600006FF05FF813050401EF2010179307100027
:10161000E31AF5F66FF09FFE13050400EFF00FA339
:10162000EF10D010130500006FF05FF663000506A1
:10163000130101FF2324810023202101232611000F
:10164000232291008324450013890500130405001B
:10165000EF20D0426380A404930600001306090023
:101660009305000013050400EFF05FCC9307100012
:10167000630CF5028320C100032481008324410010
:101680000329010013010101678000007370043019
:101690006F0000008327C400130510009387170014
:1016A0002326F4006FF01FFD8327C40093871700E3
:1016B0002326F4006FF01FFC630805066386050C03
:1016C000130101FE232C8100232A910023282101EC
:1016D000232631012324410113040500232E110088
:1016E0001309060093890500EFE0DFFE83278403DA
:1016F000130A050093040000639C070213050A0007
:10170000EFE0DFFC8320C101032481011385040085
:1017100003290101832441018329C100032A810097
:101720001301010267800000737004306F00000035
:1017300003260404630406028325C40083274400AF
:10174000B385C5002326B40063E6F50083250400B5
:101750002326B40013850900EF40805B83278403B0
:101760001307F0FF9387F7FF232CF4028327440429
:101770006384E702832744049304100093871700CF
:101780002322F4046FF09FF783270504E38A07F20E
:10179000737004306F000000832704016396070014
:1017A000930410006FF09FF513050401EF20C07C37
:1017B000E30805FEE30609FE930710002320F90065
:1017C0006FF01FFE6306050883270504638A05087A
:1017D00063840708130101FE232C8100232A910052
:1017E000232821012324410113040500232E110085
:1017F00023263101138A0500EFE0DFED8327840300
:101800001309050093040000638E07008329C400B8
:1018100093050A0013050400EFF00F8093041000F5
:101820002326340113050900EFE05FEA8320C1019C
:10183000032481011385040003290101832441014C
:101840008329C100032A810013010102678000007F
:10185000737004306F000000737004306F0000007C
:10186000E38C07FE737004306F0000006316050000
:10187000737004306F000000130101FF2324810006
:101880001304050023261100EF20104003248403D5
:10189000EF20D0428320C1001305040003248100FF
:1018A00013010101678000006316050073700430A6
:1018B0006F000000130101FF232611002324810083
:1018C00013040500EF20503C832784030324C40342
:1018D0003304F440EF20903E130504008320C10040
:1018E00003248100130101016780000063060500E5
:1018F0000325850367800000737004306F000000CB
:101900006308050497870300938747ED03A7470003
:101910006304E50403A7C7006302E50803A74701C2
:10192000630AE50603A7C7016302E50603A74702AA
:10193000630AE50403A7C7026302E50403A747039C
:10194000630AE50203A7C7036302E5026F40C033E1
:10195000737004306F000000130700001317370086
:10196000B387E70023A007006F4000321307700021
:101970006FF0DFFE130760006FF05FFE130750008B
:101980006FF0DFFD130740006FF05FFD13073000BD
:101990006FF0DFFC130720006FF05FFC13071000EF
:1019A0006FF0DFFB0325C504678000002326B50424
:1019B0006780000003450505678000006308050097
:1019C000032585031335150067800000737004300C
:1019D0006F000000630C0500832785030325C50302
:1019E0003305F5401335150067800000737004302F
:1019F0006F00000097870300938747DE03A7070067
:101A00006300070403A787006308070403A707010F
:101A10006308070403A787016308070403A70702F5
:101A20006308070403A787026308070403A70703E3
:101A3000630C070403A7870363040704678000009F
:101A40001307000013173700B387E70023A0B70080
:101A500023A2A70067800000130710006FF09FFE0D
:101A6000130720006FF01FFE130730006FF09FFD7B
:101A7000130740006FF01FFD130750006FF09FFC2D
:101A8000130770006FF01FFC130760006FF09FFBDF
:101A900097870300938787D403A747006300E50473
:101AA00003A7C7006306E50403A747016306E5042F
:101AB00003A7C7016306E50403A747026306E5041D
:101AC00003A7C7026306E50403A74703630AE50407
:101AD00003A7C7036302A704678000001307000081
:101AE00013173700B387E70023A0070067800000C3
:101AF000130710006FF0DFFE130720006FF05FFE8A
:101B0000130730006FF0DFFD130740006FF05FFD3B
:101B1000130750006FF0DFFC130770006FF05FFCDD
:101B2000130760006FF0DFFB130101FF2324810026
:101B300023229100232021011304050023261100F4
:101B40009384050013090600EF20101403274404B2
:101B50009307F0FF6314F70023220404032784048F
:101B60009307F0FF6314F70023240404EF201015FB
:101B700083278403639A07001306090093850400F2
:101B800013054402EF20802EEF20101083278404D9
:101B9000635AF004832744026386070493044402D3
:101BA0006F000002832784049387F7FF2324F40443
:101BB000832784046358F002832744026384070266
:101BC00013850400EF20403BE30E05FCEF20006886
:101BD000832784049387F7FF2324F4048327840452
:101BE000E34CF0FC9307F0FF2324F404EF20100DE6
:101BF000EF20900983274404635AF00483270401EB
:101C000063860704930404016F00000283274404E1
:101C10009387F7FF2322F404832744046358F002D8
:101C2000832704016384070213850400EF20C03476
:101C3000E30E05FCEF208061832744049387F7FFC0
:101C40002322F40483274404E34CF0FC9307F0FFC1
:101C50002322F404032481008320C1008324410053
:101C600003290100130101016F20500597F70100BE
:101C70009387078F83A6070017F701001307078DC7
:101C80000327070023A2A600636AE504130101FFEE
:101C9000232481002326110017F701001307078C66
:101CA000130405000325070083A50700938545005D
:101CB000EFE05FAD97F701009387878783A7070061
:101CC0006376F40097F7010023A487868320C10080
:101CD00003248100130101016780000017F7010050
:101CE000130787870325070083A507009385450011
:101CF0006FE05FA997F701009387878603A7070026
:101D000083A60700832747049387F7FF2322F7045E
:101D100083A7460463940700736004306780000063
:101D200063020504130101FD232E3101232A510111
:101D300023261102938A0700232481022322910281
:101D400023202103232C4101232861012326710133
:101D5000930740009309070063FAE70073700430AB
:101D60006F000000737004306F000000130B05005B
:101D70009384050013090600938B0600130A0800DC
:101D80006302082C13050006EF30105813040500F9
:101D90006302052A131929002328450313060900A5
:101DA0009305500A13050A00EF40800803C704009A
:101DB000832704031309C9FF230AE40203C70400AD
:101DC000338927011379C9FF6306070E83C71400FF
:101DD000A30AF40283C71400638E070C83C7240090
:101DE000230BF40283C724006386070C83C73400E7
:101DF000A30BF40283C73400638E070A83C7440031
:101E0000230CF40283C744006386070A83C7540087
:101E1000A30CF40283C75400638E070883C76400D1
:101E2000230DF40283C764006386070883C7740028
:101E3000A30DF40283C77400638E070683C7840072
:101E4000230EF40283C784006386070683C79400C9
:101E5000A30EF40283C79400638E070483C7A40013
:101E6000230FF40283C7A4006386070483C7B4006A
:101E7000A30FF40283C7B400638E070283C7C400B4
:101E80002300F40483C7C4006386070283C7D40019
:101E9000A300F40483C7D400638E070083C7E40063
:101EA0002301F40483C7E4006386070083C7F400BA
:101EB000A301F404130A440013050A00A301040457
:101EC0002326340323283405232A0404EFE01F8843
:101ED00013058401EFE09F8793075000B3873741D4
:101EE000232C040423288400232CF40023228402BE
:101EF00023220404232E040413860B0093050B00F5
:101F000013050900EFE0CFFD2320A40063840A003D
:101F100023A08A007370043017E901001309896255
:101F20008327090097E4010093848463638C07008E
:101F300003A7040083A7040083274704938717009F
:101F40002322F70417E701001307876083270700A0
:101F50009387170097E6010023ACF65E83A7040081
:101F6000638E070E83270900639C070083A7040084
:101F700083A7C70263E6F90097E7010023A2875E03
:101F800097E701009387075B03A7070097E6010027
:101F90009386865B8327C40283A606001307170077
:101FA00017E601002328E6582324E40463F6F6002C
:101FB00017E70100232AF75813074001B387E70208
:101FC00017E501001305C56B93050A003305F500FD
:101FD000EFE04FF8832709006388070083A7040018
:101FE00083A7470463900712832709001304100096
:101FF000638A070083A7040083A7C70263F437013D
:10200000EFE00FD9130504008320C10203248102ED
:1020100083244102032901028329C101032A81018A
:10202000832A4101032B0101832BC100130101030A
:102030006780000013050A00EF3010451304F0FF1D
:102040006FF05FFC13152600EF30102C130A05000B
:10205000E31A05D21304F0FF6FF0DFFA97E70100EF
:1020600023A087500327070093071000E31AF7F017
:1020700017E501001305C560EFE04FEB17E5010020
:1020800013054561EFE08FEA17E501001305C5610F
:10209000EFE0CFE917E5010013054562EFE00FE936
:1020A00017E501001305C562EFE04FE817EB0100EB
:1020B000130B4B6313050B00EFE04FE797EA0100AA
:1020C000938A8A6313850A00EFE04FE617E5010063
:1020D0001305C563EFE08FE517E5010013054564BF
:1020E000EFE0CFE417E501001305C564EFE00FE46E
:1020F00097E7010023A4674797E7010023AE574500
:102100006FF01FE803A7040083A604008327470499
:102110009387F7FF2322F70483A74604E39607EC8F
:10212000736004306FF05FEC130101FF2324810022
:1021300023261100232291002320210113040500EE
:102140007370043097E401009384C43F83A70400B4
:10215000639E07106318040097E7010093874740C8
:1021600003A407001309440013050900EFE0CFE6BC
:10217000832784026386070013058401EFE0CFE51F
:102180009305090017E5010013058559EFE08FDC81
:1021900097E701009387073C03A7070097E7010033
:1021A0009387473983A707001307170097E60100B5
:1021B00023A2E63A03A704009387170097E60100DD
:1021C00023AAF636630C070097E701009387473987
:1021D00003A7070003274704631C070E83A7040017
:1021E000638A070697E701009387873703A70700ED
:1021F000630287107370043003A704006318070894
:1022000017E70100130787358326070083A606001A
:102210006392060A1307F0FF97E6010023AAE6304F
:1022200003A704006308070203A707000327470466
:102230006302070203A7070083A60700832747045A
:102240009387F7FF2322F70483A7460463940700CC
:10225000736004308320C100032481008324410083
:1022600003290100130101016780000097E70100C5
:102270009387072F03A7070083A707008327470437
:10228000938717002322F7046FF0DFEC83A6070083
:1022900003A7070003A746041307170023A2E604B9
:1022A00017E701001307872B8326070083A6060084
:1022B000E38206F6032707000327C7000327C700AA
:1022C0000327470097E6010023A4E6266FF05FF599
:1022D00003A7070083A60700832747049387F7FF18
:1022E0002322F70483A74604E39A07EE73600430C1
:1022F0006FF0DFEE97E701009387472383A707007E
:1023000063860700737004306F00000003248100AF
:102310008320C1008324410003290100130101012E
:102320006FE00FA76304050C17E7010013074723AD
:1023300083260700930700006386A60A130101FFA6
:10234000232611002324810023229100737004307E
:1023500097E601009386061F83A70600638C07009B
:102360000326070083270700832746049387170067
:102370002322F60483A706009304050003244501E5
:10238000638807008327070083A747046394070631
:1023900097E701009387871C83A70700638C870654
:1023A00097E701009387471B83A70700638487068D
:1023B00097E70100938707386306F40497E7010065
:1023C00093870736630CF402930710008320C10043
:1023D00003248100832441001385070013010101B8
:1023E0006780000013850700678000007370043069
:1023F0006F000000EFF01F906FF09FF9930740000F
:102400006FF0DFFC83A7840293B717009387270040
:102410006FF0DFFB930720006FF05FFB73700430F9
:1024200097E701009387071203A7070063160702C7
:102430006304050483A707000325C502638C070016
:1024400097E701009387C71103A7070003274704F5
:10245000631C07026780000017E70100130747109D
:10246000832607000327070003A746041307170066
:1024700023A2E604E31005FC17E701001307470E4B
:10248000032507006FF01FFB03A7070083A60700C3
:10249000832747049387F7FF2322F70483A7460483
:1024A000E39A07FA7360043067800000130101FFAC
:1024B000232481001304050023261100EFE08FA1DF
:1024C0006318040097E701009387870903A40700B6
:1024D0000324C402EFE08F9F8320C1001305040092
:1024E000032481001301010167800000930740006D
:1024F00063F6B700737004306F000000130101FE33
:10250000232C8100232E1100232A9100232821014E
:102510002326310123244101130405007370043084
:1025200017E90100130909028327090063920710C4
:102530006300041283270405638EF50A17E7010080
:102540001307070263F0B70283260700638E861223
:10255000032707008324C702B3B4950093C4140073
:102560006F00000183240700B384844093B41400F7
:102570000327C4026386E70E832784012328B4045B
:1025800063C8070093075000B385B740232CB400FD
:1025900093172700B387E7000327440197E9010059
:1025A0009389090E93972700B387F9006310F70406
:1025B000130A440013050A00EFE00FA217E7010019
:1025C000130787F88327C402032707006376F70001
:1025D00017E70100232AF7F613074001B387E70244
:1025E00093050A003385F900EFE0CF966384040079
:1025F000EFD01FFA83270900638C070097E70100DB
:10260000938707F683A7070083A74704639E070401
:102610008320C10103248101832441010329010195
:102620008329C100032A8100130101026780000091
:1026300097E701009387C7F203A7070083A7070066
:1026400083274704938717002322F704E31404EE3B
:1026500097E701009387C7F003A407006FF09FED91
:102660002326B4026FF05FF1032481018320C101AE
:1026700083244101032901018329C100032A810028
:10268000130101026FF00FE7930400006FF05FEE9B
:10269000630A0508130101FE232A910097E4010053
:1026A000938404EC83A70400232E1100232C8100C3
:1026B00023282101232631016388A7047370043085
:1026C00017E90100130909E883270900638C070053
:1026D00003A7040083A704008327470493871700F8
:1026E0002322F7040327450197E701009387870416
:1026F000630EF702832709006388070083A704009D
:1027000083A74704639E07088320C1010324810136
:1027100083244101032901018329C100130101021E
:1027200067800000737004306F000000832785020B
:1027300017E70100130787FDE38EE7FAE39C07FA2A
:10274000930945001304050013850900EFE0CF88C5
:1027500017E70100130747DF8327C4020327070099
:102760006376F70017E701002320F7DE1307400127
:10277000B387E70217E50100130585F0938509008B
:102780003305F500EFD01FFD83A704000327C40223
:1027900083A7C702E360F7F6EFD09FDF6FF09FF5E6
:1027A000032481018320C101832441010329010104
:1027B0008329C100130101026FF0CFD36302050624
:1027C000130101FE232C8100232A910023282101DB
:1027D00013040500232E110023263101EFD09FEFB3
:1027E0000327440197E701009387C7F41309050005
:1027F00093040000630AF70213050900EFD01FEDF0
:102800008320C101032481011385040003290101F0
:10281000832441018329C100130101026780000064
:10282000737004306F0000008327840217E50100F5
:102830001305C5EDE382A7FCE39007FC97E70100D1
:102840009387C7CE83A707006394070697E7010025
:10285000938707D183A707008324C4029309440008
:1028600083A7C70213850900B3B4F400EFD0DFF6E5
:1028700017E70100130747CD8327C402032707008A
:1028800093C414006376F70017E70100232EF7CAFC
:1028900013074001B387E70217E50100130545DE82
:1028A000938509003305F500EFD0DFEA6FF0DFF420
:1028B00093058401EFD01FEA6FF01FF4130101FEAE
:1028C00037150000232E1100232C8100232A9100AC
:1028D00023282101232631012324410123225101F0
:1028E000EF308022630605249304050013050006DB
:1028F000EF3080211304050063000528371600001F
:102900009305500A2328950213850400EF304052A6
:1029100083240403B71700009387C7FFB384F40030
:10292000B7474C459387974493094400232AF40200
:1029300013850900230C0402A301040423260402C6
:1029400023280404232A0404EFD05FE01305840144
:10295000EFD0DFDF93075000232C040493F4C4FF6F
:1029600023288400232CF40023228402232204043D
:10297000232E04041306000097150000938585EAB2
:1029800013850400EFD0DFD52320A400737004303A
:1029900017E90100130909BB8327090097E4010027
:1029A000938404BC638C070003A7040083A704007E
:1029B00083274704938717002322F70417E70100B2
:1029C000130707B9832707009387170097E60100CD
:1029D00023A0F6B883A704006388070A83270900A9
:1029E000639C070083A7040083A7C70263960700C0
:1029F00097E7010023A687B697E70100938787B37F
:102A000083A7070097E60100938606B40327C40254
:102A100083A606009387170017E60100232CF6B063
:102A20002324F40463F6E60097E7010023AEE7B041
:102A300093172700B387E7009397270017E5010056
:102A4000130505C43305F50093850900EFD09FD029
:102A5000832709006388070083A7040083A747042E
:102A6000639A070E832709006384070083A7040085
:102A7000EF201006930710006304F512631A050A8D
:102A8000737004306F00000097E7010023AA87AC41
:102A90000327070093071000E310F7F617E501007E
:102AA000130505BEEFD09FC817E50100130585BECD
:102AB000EFD0DFC717E50100130505BFEFD01FC733
:102AC00017E50100130585BFEFD05FC617E50100CC
:102AD000130505C0EFD09FC597EA0100938A8AC00D
:102AE00013850A00EFD09FC417EA0100130ACAC079
:102AF00013050A00EFD09FC317E50100130505C1B8
:102B0000EFD0DFC217E50100130585C1EFD01FC26A
:102B100017E50100130505C2EFD05FC197E701007B
:102B200023AE57A397E7010023A847A36FF0DFEC7C
:102B30008320C10103248101832441010329010170
:102B40008329C100032A8100832A41001301010265
:102B50006780000003A7040083A6040083274704BE
:102B60009387F7FF2322F70483A74604E39C07EE2D
:102B7000736004306FF01FEF032481018320C101D3
:102B8000032901018329C100032A8100832A41000E
:102B90001385040083244101130101026F30C00E2C
:102BA000737004309307F0FF17E701002322F798B2
:102BB0000324810197E7010023A6A7988320C10180
:102BC00083244101032901018329C100032A8100D3
:102BD000832A410097E7010023AA07961301010207
:102BE0006FD05F807370043097E7010023AC0794C7
:102BF0006FD09F9117E701001307479383270700C2
:102C0000938717002320F70067800000737004305B
:102C100097E701009387079303A70700631807024C
:102C200017E70100130787920325070083A7070012
:102C3000638C070097E701009387879203A707003B
:102C400003274704631407026780000017E70100A9
:102C500013070791832607000327070003A74604ED
:102C60001307170023A2E6046FF09FFB03A70700DA
:102C700083A60700832747049387F7FF2322F704DF
:102C800083A74604E39207FC73600430678000006A
:102C9000130101FF2326110023248100EFD09FA3FD
:102CA00097E701009387878A03A40700EFD01FA24C
:102CB0008320C100130504000324810013010101D6
:102CC0006780000097E701009387878803A50700C6
:102CD00067800000130101FD2326110223248102D5
:102CE0002322910223202103232E3101232C410191
:102CF000232A5101232861012326710197E701004E
:102D00009387C78283A70700639A070617E7010026
:102D10001307C783832707009387170097E60100EF
:102D200023A6F682832A0700638A0A0A97E701002E
:102D30009387078083A707009304000063FEFA0AC5
:102D400097E901009389C99317EA0100130A4A81A0
:102D500083270A009306100003A7C70293172700D2
:102D6000B387E70093972700B389F90083A7090089
:102D700063F4F602930410006F00000297D701007D
:102D80009387077C83A707009304000093871700AD
:102D900017D701002326F77A97D701009387077A80
:102DA00083A7070063840700930410008320C102F7
:102DB00003248102138504000329010283244102B4
:102DC0008329C101032A8101832A4101032B0101C7
:102DD000832BC100130101036780000017D4010099
:102DE0001304C4778327040083A707006388070CB4
:102DF000737004306F00000017D4010013040476D0
:102E000097E901009389C98717DA0100130A4A7507
:102E100017DB0100130B4B738327040083A7070004
:102E2000638007088327040083A7C70003A9C7009E
:102E300083274900930B490013850B0063EAFA06C8
:102E4000EFD09F99832789021305890163840700C6
:102E5000EFD09F988327C90203270B0093850B00AF
:102E6000139527003305F500131525003385A900B8
:102E70006376F70017D701002328F76CEFD09F8DFA
:102E800083270A000327C90283A7C702E366F7F86E
:102E9000832704009304100083A70700E39407F836
:102EA0009307F0FF17D701002324F7686FF05FEA5C
:102EB00017D70100232EF7666FF09FE917D701009F
:102EC00013078769832704000327070097D60100AB
:102ED00023A6E66817D701002320F76897D70100DB
:102EE0009387876583A707009387170017D701008B
:102EF0002324F7648327040083A70700639A07004D
:102F00009307F0FF17D701002324F7626FF01FE249
:102F10008327040083A7C70083A7C70083A74700B0
:102F200017D701002326F7606FF05FE097D7010005
:102F30009387C75F03A70700631607007370043009
:102F40006F000000130101FE232E1100232C8100CD
:102F5000232A910023282101232631012324410122
:102F600023225101232061017370043097D40100A2
:102F70009384445D03A704006310071203A70700AE
:102F80001307F7FF97D6010023A2E65A83A707008D
:102F9000639E070A97D701009387875B83A7070083
:102FA0006386070A97DA0100938A8A6D17DA0100AF
:102FB000130A8A5917D901001309895A9309100075
:102FC0006F00C0013385EA00EFD0CFF883270900F6
:102FD0000327C40283A7C7026374F70683A7CA083E
:102FE0006380070E83A78A0903A4C7001305840121
:102FF000EFD08FFE130B440013050B00EFD0CFFD75
:103000008327C40283260A0093050B00139527002B
:103010003305F50013152500130705003385AA00B5
:10302000E3F2F6FA17D701002320F752EFD08FF220
:10303000832709000327C40283A7C702E360F7FAC6
:1030400097D7010023AC374F6FF05FF913040000EE
:1030500083A70400638C070097D70100938747502C
:1030600083A7070083A74704639807041305040098
:103070008320C1010324810183244101032901012B
:103080008329C100032A8100832A4100032B010008
:10309000130101026780000017D701001307474C96
:1030A000832607000327070003A74604130717001A
:1030B00023A2E6046FF09FECEFE0DFC36FF01FFB8D
:1030C00017D401001304C44783270400638C07024C
:1030D000832704001309100063860702EFF09FBFE7
:1030E0006306050097D7010023AA2745832704001C
:1030F0009387F7FF17D701002324F74483270400A1
:10310000E39E07FC97D701009387474303A7070077
:1031100093071000E31CF7F2EFD08FC713041000E1
:103120006FF01FF3630405026396050073700430AB
:103130006F00000017D701001307473F83270700E0
:10314000638A0700737004306F00000073700430EE
:103150006F000000130101FF2324810023261100CA
:1031600083260700032705009386160017D6010063
:10317000232ED63A97D601009386463D83A60600B5
:103180003304B7002320850063F0E6046372E40291
:1031900063F0860297D701009387873C03A5070059
:1031A00013054500EFD04FE313050400EFE01FAC1B
:1031B000EFF0DFD7630E05008320C10003248100F8
:1031C0001301010167800000E366E4FC6FF05FFC1F
:1031D000032481008320C100130101016FD04FBB84
:1031E000630E050017D70100130747348327070034
:1031F00063880700737004306F0000006FD04FB910
:10320000130101FF23261100232481000327070057
:10321000930705001307170097D6010023A8E6308F
:1032200097D601009386C63317D7010013070732DC
:103230000327070003A506003304F7001305450024
:10324000EFD08FD913050400EFE05FA2EFF01FCE9F
:10325000631A0500032481008320C10013010101CA
:103260006FD00FB38320C10003248100130101013B
:1032700067800000130101FF232481002326110031
:1032800097D701009387872A83A7070013040000BC
:103290009387170017D70100232AF72897D7010033
:1032A0009387072B83A7070063ECF50E17DE010059
:1032B000130E8E4297D201009382C23B130400008A
:1032C00013070000930F10001303500A6F00C00093
:1032D000130ECEFE6386C21183278EFF930507006F
:1032E000E38807FE8327CEFF83A74700232EFEFE39
:1032F0006388C72103AFC70083A747003307E500F2
:10330000930E0000232EFEFE6380C70983A8C7002A
:1033100093874803232017012322F70083A78804FB
:103320002326F7012324F70083A7C8022328F700E8
:1033300083A70805232C0700232AF70003A8080306
:1033400083470800639A670693070800938717006E
:1033500083C60700B3850741E38A66FE93D525003F
:103360009395050193D50501231EB700938E1E008A
:1033700013070702630C1F058327CEFF83A74700AF
:10338000232EFEFEE394C7F983274E00232EFEFE74
:103390006FF0DFF7330464006304060023200600A7
:1033A000EFF0DFB8130504008320C100032481007F
:1033B000130101016780000093050000231EB70080
:1033C000938E1E0013070702E3181FFB3304D4017A
:1033D00013175400130ECEFE93050700E39EC2EFB1
:1033E00097D701009387871703AE070083270E0046
:1033F000639E071097D701009387071603AE070057
:1034000083270E006392071C17DE0100130E4E2760
:1034100083270E0A6398072683274E0BE38E07F651
:1034200083278E0B97DE0100938E4E3183A74700D2
:1034300017D701002322F730638CD73D83AFC70035
:1034400083A747003307B5001303000097D6010098
:1034500023A4F62E130F3000930220009308500A85
:103460006388D70903A5C700930745032320A70056
:103470002322F700832785042326E7012324F7006E
:103480008327C5022328F70083278502638407006A
:103490002326570083270505232C0700232AF7003E
:1034A0000328050383470800639C1733930708002C
:1034B0009387170083C60700B3850741E38A16FF89
:1034C00093D525009395050193D50501231EB700DB
:1034D0001303130013070702E38EAFEA83278E0B53
:1034E00083A7470097D6010023A8F624E39CD7F7CB
:1034F00083270E0C97D6010023A0F6246FF09FF6C9
:1035000083274E00232EFEFE6FF0DFDE83274E0062
:10351000130F8E0083A647002322DE00638CE62D66
:10352000B307E50003A7460083A2C600930E000080
:103530002322EE00930F20001303500A6300EF08CC
:103540008328C7001387480323A0170123A2E7009D
:1035500003A7880423A6F70123A4E70003A7C80252
:1035600023A8E70003A7080523AC070023AAE70068
:1035700003A8080303470800631A6722130708001B
:103580001307170083460700B3050741E38A66FE69
:1035900093D525009395050193D50501239EB7008A
:1035A000938E1E0093870702638C122183264E00A0
:1035B00003A746002322EE00E314EFF80327CE0012
:1035C0002322EE006FF0DFF783274E00130F8E00EB
:1035D00083A747002322FE006388E72183A2C70058
:1035E00083A74700B305B500930E00002322FE0019
:1035F000930F20001303500A6300FF0883A8C7003D
:103600009387480323A0150123A2F50083A788040C
:1036100023A6F50123A4F50083A7C80223A8F5007B
:1036200083A7080523AC050023AAF50003A8080317
:103630008347080063946714930708009387170073
:1036400083C6070033870741E38A66FE13572700C6
:103650001317070113570701239EE500938E1E00E1
:10366000938505026386121383274E0083A74700C4
:103670002322FE00E314FFF88327CE002322FE005E
:103680006FF0DFF783274E0A17DF0100130FCF0912
:1036900083A7470017D701002326F7086382E7179F
:1036A00083A2C70083A74700B305B500930E0000AF
:1036B00017D701002328F706930F40001303500A81
:1036C0006382E70983A8C7009387480323A01501F5
:1036D00023A2F50083A7880423A6F50123A4F500FF
:1036E00083A7C80223A8F50083A7080523AC05001B
:1036F00023AAF50003A8080383470800639C670416
:10370000930708009387170083C607003387074194
:10371000E38A66FE135727001317070113570701A3
:10372000239EE500938E1E0093850502638E12038F
:1037300083274E0A83A7470017D701002324F7FEEB
:10374000E392E7F98327CE0A17D70100232CF7FC71
:103750006FF05FF713070000239EE500938E1E00B5
:1037600093850502E39612FD83274E0B3304D401A3
:1037700093155400E38207C26FF09FCA130700003D
:10378000239EE500938E1E0093850502E39E12EDB5
:1037900017DE0100130ECEEE83270E0A3304D40188
:1037A00093155400E38A07C66FF0DFED9305000020
:1037B000239EB700938E1E0093870702E39812DFC3
:1037C00097D70100938747D903AE07003304D4018C
:1037D0009315540083270E00E38807C26FF0DFDEE5
:1037E000930500006FF09FCE8327CE002322FE00BA
:1037F0006FF0DFDE8326CE002322DE006FF05FD283
:103800008327CE0A17D70100232EF7F06FF05FE968
:1038100083270E0C17D701002320F7F26FF01FC289
:10382000130101FD2322910223202103232E3101C4
:10383000232C4101232A51012328610123267101F0
:10384000232611022324810297D90100938909CEEE
:1038500017D901001309C9E217DA0100130A8ACE49
:1038600097DA0100938ACACF97DB0100938B4BCE86
:1038700097D40100938404CE130B10006F00000254
:1038800083A709000324090A9387170017D70100AB
:10389000232EF7C8EFF08FE9631E040083A704000E
:1038A000E39007FE83270900E37AFBFEEFC05FCEBB
:1038B0006FF0DFFE7370043083270A00639E0704F5
:1038C0008327C90A03A4C70013054400EFC0DFF033
:1038D00083A70B009387F7FF17D70100232AF7C6AA
:1038E00083A704009387F7FF17D701002324F7C6A7
:1038F00083270A006388070083A70A0083A7470479
:103900006398070203250403EF2000381305040021
:10391000EF2080376FF09FF803A70A0083A70A0003
:1039200083274704938717002322F7046FF05FF97A
:1039300003A70A0083A60A00832747049387F7FF9B
:103940002322F70483A74604E39E07FA736004303A
:103950006FF05FFB97D70100938747BD83A70700F0
:103960006396070E130101FF2326110097D701006C
:1039700023A607BC17D70100130787BE83270700BC
:10398000B7A6A5A59386565A83A7070383A5070064
:10399000639ED50003A64700631AB60083A687007E
:1039A0006396C60083A7C700638AD7000325070074
:1039B0008325070093854503EF30900997D60100D2
:1039C000938686B803A6060017D70100130747CBD6
:1039D0006F00000283A706006382070883A7060022
:1039E0009387F7FF17D601002320F6B603A606003B
:1039F00093172600B387C70093972700B307F700F4
:103A000083A70700E38807FC03A606009317260098
:103A1000B387C70093972700B305F70083A6450037
:103A200093878700B307F70083A6460023A2D5003B
:103A3000638AF60283A7C6008320C10017D701005E
:103A40002320F7B2130101016780000093071000E3
:103A500017D701002324F7AE67800000737004308D
:103A60006F000000930740013306F60283A646006C
:103A70003307C7002322D7006FF0DFFB130101FEDD
:103A800023282101232E1100232C8100232A9100B9
:103A900023263101130905007370043097D4010007
:103AA000938444AA83A7040017D40100130444ABF1
:103AB000639C070C6314090003290400930949005F
:103AC00013850900EFC05FD1832789026386070051
:103AD00013058901EFC05FD09385090017D5010058
:103AE000130545C5EFC01FC783A7040063880700FF
:103AF0008327040083A747046394070A83270400ED
:103B00006384270D83A70400638207067370043063
:103B100083A704006398070E97D70100938707A433
:103B200003A70700032707006310070C9307F0FFA4
:103B300017D70100232EF79E83A70400638807028E
:103B40008327040083A74704638207020327040036
:103B500083260400832747049387F7FF2322F70473
:103B600083A7460463940700736004308320C10177
:103B70000324810183244101032901018329C10018
:103B8000130101026780000003270400832704005B
:103B900083274704938717002322F7046FF09FF1D0
:103BA0000327040083260400832747049387F7FF35
:103BB0002322F70483A74604E39207F473600430DA
:103BC00083270400E39027F583A704006382070698
:103BD00097D701009387879583A707006388070A13
:103BE000737004306F00000083A7070083A7C7002D
:103BF00083A7C70083A7470017D70100232AF7929E
:103C00006FF09FF3032704008327040083274704F2
:103C1000938717002322F70497D70100938707940F
:103C200003A7070003270700E30207F06FF0DFFB9D
:103C300097D701009387C79117D70100130747A4AF
:103C400083A707000327470B6314F7028320C101F2
:103C50000324810197D7010023A407908324410105
:103C6000032901018329C1001301010267800000BB
:103C7000032481018320C10183244101032901011F
:103C80008329C100130101026FF0DFCC03248101FD
:103C90008320C10183244101032901018329C1003B
:103CA000130101026FC0DF8E6306050A130101FFD5
:103CB0002322910097D401009384848A2320210138
:103CC0001389050083A50400232611002324810005
:103CD00093858501EFC01FAB03A5040013054500C4
:103CE000EFC09FAF9307F0FF630AF90697D7010073
:103CF0009387C78503A4070003A7040083A70700D1
:103D00003304240123228700636EF40697D7010051
:103D10009387C78403A5070083A504009385450006
:103D2000EFC05FA697D701009387878083A707001E
:103D30006376F40097C7010023AC877E8320C1001F
:103D400003248100832441000329010013010101A0
:103D500067800000737004306F00000083A50400CA
:103D6000032481008320C100832441000329010032
:103D700017D501001305059C93854500130101012A
:103D80006FC05F9D97C701009387077D03A507005C
:103D90000324810083A504008320C1008324410003
:103DA0000329010093854500130101016FC09F9D08
:103DB000630E050097C701009387477783A7070025
:103DC000639A0700737004306F0000007370043052
:103DD0006F000000130101FF2322910097C401002E
:103DE0009384047803A704009387050083A5040047
:103DF000B7060080B3E7D7002326110023248100F3
:103E0000232CF7009385850113040600EFC09F94CF
:103E100003A5040013054500EFC01F9C9307F0FFA6
:103E20006304F40297C701009387477203A5070054
:103E30008320C100832441003305850003248100D1
:103E4000130101016FD09FE283A5040003248100C8
:103E50008320C1008324410017D501001305858DFF
:103E600093854500130101016FC0DF8E6308050AC9
:103E7000130101FF2322910097C401009384446E33
:103E8000232021011389050083A5040023261100A6
:103E9000232481009385850113040600EFC09F8BC6
:103EA00003A5040013054500EFC01F9393071000FE
:103EB000630AF40697C701009387476903A40700C4
:103EC00003A7040083A707003304240123228700EB
:103ED000636EF40697C701009387476803A5070040
:103EE00083A5040093854500EFC0DF8997C70100D3
:103EF0009387076483A707006376F40097C70100E0
:103F000023A887628320C100032481008324410009
:103F10000329010013010101678000007370043060
:103F20006F00000083A50400032481008320C100EA
:103F3000832441000329010017C501001305857F73
:103F400093854500130101016FC0DF8097C7010011
:103F50009387876003A507000324810083A50400DD
:103F60008320C1008324410003290100938545007B
:103F7000130101016FC01F81130101FF23261100EE
:103F800023248100232291008327C50003A4C700B6
:103F90006304040A9304840113850400EFC0DF83E3
:103FA00097C701009387875883A70700639A07087C
:103FB0009304440013850400EFC01F8297C70100DB
:103FC000938787580327C40283A7070063F6E70097
:103FD00097C7010023AAE75693172700B387E70086
:103FE0009397270017C50100130585699385040081
:103FF0003305F500EFC00FF697C7010093874756CA
:1040000083A707000327C4021305000083A7C70284
:1040100063FAE7009307100017C701002320F75247
:10402000130510008320C100032481008324410074
:104030001301010167800000737004306F000000FD
:104040009385040017C501001305456CEFC08FF080
:104050006FF09FFA97C701009387474D83A707002A
:1040600063960700737004306F000000130101FFB6
:10407000232611002324810023229100B70700800A
:104080000324C500B3E7F5002320F5006308040806
:10409000EFC08FF49304440013850400EFC0CFF306
:1040A00097C701009387474A0327C40283A70700E5
:1040B00063F6E70097C7010023A8E7489317270096
:1040C000B387E7009397270017C501001305455BE9
:1040D0003305F50093850400EFC0CFE797C70100D3
:1040E0009387074883A707000327C402130500002E
:1040F00083A7C70263FAE7009307100017C7010000
:10410000232EF742130510008320C10003248100F1
:1041100083244100130101016780000073700430A3
:104120006F0000006304050297C701009387C74032
:1041300003A7070097C701009387474183A707009C
:104140002320E5002322F50067800000737004300F
:104150006F0000006304050E638E050C130101FF60
:1041600023261100232481001307050073700430F7
:1041700097C801009388083D83A708006380070261
:1041800097C701009387C73D83A6070083A7070051
:1041900083A746049387170023A2F60417C30100E0
:1041A0001303C33A83A70500032603009306F0FF19
:1041B000130400006388D70417CE0100130ECE3716
:1041C00003250E0003280700832647006306A80086
:1041D000130410006378D6023308D640130410008D
:1041E0006372F80203250E00B387C740032603005D
:1041F000B387D70023A0F5002320A7002322C70000
:104200001304000083A70800638C070097C7010010
:104210009387073583A7070083A7470463940702A2
:10422000130504008320C100032481001301010150
:1042300067800000737004306F00000073700430FA
:104240006F000000EFD01FAB6FF09FFD93071000D1
:1042500017C701002324F72E6780000063060500BE
:104260000325C50467800000130500006780000077
:10427000630405002326B5046780000097C701008A
:104280009387072E03A507006780000097C70100EA
:104290009387472B83A7070013051000638C070043
:1042A00097C701009387872803A5070013351500DA
:1042B0001315150067800000630C0508130101FE4B
:1042C000232A910097C401009384842983A70400C2
:1042D000232E1100232C81002328210123263101C4
:1042E0000327C50283A7C7026376F70483278501E6
:1042F00063CC070083A7040083A6C702930750007E
:10430000B387D740232CF50093172700B387E70026
:104310000327450117C90100130989369397270020
:10432000B307F9006308F70283A7040083A7C70255
:104330002326F5028320C101032481018324410146
:10434000032901018329C1001301010267800000D4
:1043500067800000930945001304050013850900D8
:10436000EFC08FC783A7040017C701001307C71D3D
:104370000327070083A7C7022326F4026376F7000A
:1043800017C701002322F71C139527003305F500FA
:1043900003248101131525008320C10183244101D9
:1043A000938509003305A9008329C1000329010170
:1043B000130101026FC00FBA63060502130101FF6A
:1043C00023261100232481002322910097C7010096
:1043D0009387071903A40700630AA40073700430CD
:1043E0006F0000001305000067800000832744056C
:1043F00063960700737004306F0000008326C402C8
:10440000032704059387F7FF232AF4046384E60057
:10441000638E0700130500008320C1000324810080
:1044200083244100130101016780000093044400CC
:1044300013850400EFC04FBA8327040517C7010096
:104440001307871083260700130750003307F74030
:104450002326F402232CE40063F6F60017C70100BC
:104460002324F70E13074001B387E70217C50100A5
:1044700013050521938504003305F500EFC08FADCA
:10448000130510006FF05FF97370043097C70100D7
:104490009387470B83A707006380070297C7010034
:1044A0009387070C03A7070083A707008327470408
:1044B000938717002322F7046780000097C7010045
:1044C0009387470883A70700638C070297C70100FB
:1044D0009387070903A7070003274704630207021E
:1044E00003A7070083A60700832747049387F7FFE6
:1044F0002322F70483A74604639407007360043003
:104500006780000097C701009387870503A607000F
:1045100083A6070003A707009307500083A6C602DF
:1045200003258601B387D740232CF700678000005E
:1045300097C701009387C70203A70700630A070014
:1045400083A6070003A746051307170023AAE6045E
:1045500003A5070067800000130101FD232021034C
:10456000232611022324810223229102232E3101CA
:10457000130905007370043097C40100938484FC10
:1045800083A7040017C40100130484FD639E070A77
:104590008327040083A78705639A07008327040005
:1045A0001307100023AEE704639A050E83A70400E7
:1045B000638807008327040083A74704639A0714CE
:1045C0007370043083A704006394070683270400F4
:1045D00003A5870563080500630209048327040017
:1045E00023AC07048327040023AE070483A7040039
:1045F000638807008327040083A7470463920706A4
:104600008320C10203248102832441020329010281
:104610008329C101130101036780000003270400FF
:10462000832787059387F7FF232CF7046FF09FFB01
:104630000327040083270400832747049387170078
:104640002322F7046FF09FF8032704008327040058
:1046500083274704938717002322F7046FF05FF343
:104660000327040083260400832747049387F7FF6A
:104670002322F70483A74604E39407F87360043009
:104680008320C10203248102832441020329010201
:104690008329C10113010103678000000325040081
:1046A0002326B10013054500EFC00F938325C100F9
:1046B0009307F0FF6380F50897C70100938707E928
:1046C00083A907000327040083A70700B389B90063
:1046D0002322370163ECF90697C70100938707E8A7
:1046E00003A507008325040093854500EFC08F894B
:1046F00097C701009387C7E383A7070063F6F90014
:1047000097C7010023A637E3EFB09FE86FF01FEAD9
:104710000327040083260400832747049387F7FFB9
:104720002322F70483A74604E39C07E87360043060
:104730006FF01FE98325040017C50100130585FFED
:1047400093854500EFC00F816FF01FFC97C70100F4
:10475000938787E003A50700832504009385450020
:10476000EFC04F826FF05FFA130101FD2320210398
:10477000232E3101232611022324810223229102B8
:10478000232C41011389050093090600737004303E
:1047900097C40100938404DB83A7040017C40100BD
:1047A000130404DC639C0714032704009307200010
:1047B0000327C7056304F702832704001345F5FFA9
:1047C00003A787053375E50023ACA70483270400FE
:1047D0001307100023AEE704639A060A83A70400B8
:1047E000638807008327040083A7470463940716A0
:1047F0007370043083A70400639E07066388090072
:104800008327040083A7870523A0F900032704005A
:1048100093071000130500000327C705630EF70078
:10482000832704001349F9FF1305100003A7870528
:104830003379E90023AC27058327040023AE07045E
:1048400083A70400638807008327040083A7470425
:104850006392070C8320C102032481028324410256
:10486000032901028329C101032A810113010103E4
:104870006780000003270400832704008327470480
:10488000938717002322F7046FF05FF703250400D6
:104890002326D10013054500EFB01FF48326C10085
:1048A0009307F0FF638AF60C97C70100938707CA46
:1048B00003AA07000327040083A70700330ADA00CE
:1048C000232247016368FA0C97C70100938707C941
:1048D00003A507008325040093854500EFB09FEAF8
:1048E00097C701009387C7C483A707006370FA0ABC
:1048F00097C7010023AE47C36F0040090327040098
:104900008327040083274704938717002322F70493
:104910006FF09FE9032704008326040083274704E0
:104920009387F7FF2322F70483A74604E39407F253
:10493000736004308320C102032481028324410276
:10494000032901028329C101032A81011301010303
:1049500067800000032704008326040083274704A0
:104960009387F7FF2322F70483A74604E39207E81F
:10497000736004306FF0DFE78325040017C5010082
:10498000130545DB93854500EFB0DFDCEFB05FC07A
:104990006FF0DFE497C70100938707BC03A507000A
:1049A0008325040093854500EFB0DFDD6FF01FFE27
:1049B000630A050C130101FF232611002324810043
:1049C00023229100232021017370043097C4010039
:1049D000938444B783A704006396070863860600A0
:1049E0008327850523A0F600930706009306200081
:1049F0000326C505232ED5041387050013040500DF
:104A00006382D70A63F4F608930530006388B70021
:104A1000930540006396B700630CD610232CE40482
:104A200093071000630CF6081304100083A704001A
:104A3000638C070097C70100938787B283A707009D
:104A400083A7470463980706130504008320C10069
:104A50000324810083244100032901001301010183
:104A60006780000097C70100938787AF03A70700FF
:104A700083A7070083274704938717002322F7049F
:104A80006FF0DFF5737004306F00000093061000C4
:104A9000E398D7F88327850533E7B700232CE5048F
:104AA0006FF01FF88327850593871700232CF504E3
:104AB0006FF01FF7EFD00FA46FF01FF91309440038
:104AC00013050900EFB05FD117C701001307C7A78F
:104AD0008327C402032707006376F70017C7010086
:104AE0002324F7A613074001B387E70217C5010087
:104AF000130505B9930509003305F500EFB09FC50F
:104B00008327840263860700737004306F000000FF
:104B100097C701009387C7A483A707000327C40290
:104B200083A7C702E3F2E7F0EFB09FA66FF0DFEFD5
:104B3000130400006FF09FEF63080508130101FEE6
:104B4000232C8100232A91002328210123263101CF
:104B50002324410123225101232E11009309070030
:104B6000138A060093040600138905001304050048
:104B7000EFB05FB6930A050063060A008327840539
:104B80002320FA000327C40593072000232EF404F2
:104B90006380F40463FA9710930630006388D400AE
:104BA000930640006396D400630CF70E232C240573
:104BB000930710006312F70A8327840263820702B7
:104BC000737004306F000000737004306F000000D9
:104BD0008327840593871700232CF4046FF05FFD6F
:104BE00097C701009387879483A707006390070AFC
:104BF0009304440013850400EFB01FBE17C70100E3
:104C0000130787948327C402032707006376F700FE
:104C100017C70100232AF79213074001B387E70261
:104C200017C501001305C5A5938504003305F500DC
:104C3000EFB05FB297C701009387879283A7070001
:104C40000327C40283A7C70263F8E700638609004D
:104C50009307100023A0F9001304100013850A0025
:104C6000EFB0DFA6130504008320C10103248101F6
:104C700083244101032901018329C100032A810002
:104C8000832A41001301010267800000930584011B
:104C900017C50100130585A7EFB0DFAB6FF09FF9D3
:104CA000130400006FF09FFB93071000E392F4F0F1
:104CB0008327840533E92701232C24056FF05FEF58
:104CC000630A050E130101FE232C8100232A9100A3
:104CD0001304050023282101232E1100232631016E
:104CE00093840500EFB01F9F930720008326C4051F
:104CF000232EF404832784051307100013090500ED
:104D000093871700232CF4046396E6088327840214
:104D100063860700737004306F00000097C70100BE
:104D20009387C78083A70700639A07089309440005
:104D300013850900EFB05FAA17C701001307C780EA
:104D40008327C402032707006376F70017B7010023
:104D5000232CF77E13074001B387E70217C5010034
:104D600013050592938509003305F500EFB09F9E6A
:104D700097B701009387C77E83A707000327C40264
:104D800083A7C70263F8E700638604009307100057
:104D900023A0F400032481018320C1018324410165
:104DA0008329C10013050900032901011301010230
:104DB0006FB0DF91737004306F00000093058401C1
:104DC00017C5010013058594EFB0DF986FF05FFA07
:104DD00093070500630805067370043017B70100D8
:104DE0001307477683260700639E060203A6C705BE
:104DF00093062000130500006316D60023AE0704B7
:104E00001305100083270700638C070097B7010084
:104E10009387077503A7070003274704631C07024E
:104E20006780000097B601009386867303A606008C
:104E300083A6060083264604938616002322D60402
:104E40006FF0DFFA97B701009387877183A7070098
:104E50006FF09FF803A7070083A607008327470486
:104E60009387F7FF2322F70483A74604E39A07FA00
:104E70007360043067800000130101FB232291045A
:104E800023202105232C4103232A510323286103D6
:104E9000232671032326110423248104232E3103A6
:104EA00023248103232291032320A10317B90100A6
:104EB0001309096C17BB0100130BCB6A97B40100EF
:104EC0009384846A97BA0100938A4A6A130A10008D
:104ED000930B90008327090003A7070063060716BA
:104EE00083A7C70083A90700EFD0DFD0EFD01FD280
:104EF00083270B00130C05006368F50C97B70100BE
:104F000023A2A766130600006376352303A50400D9
:104F1000B3858941EFC05FC1EFE04F81630605169D
:104F200003A504009306000013060000930581000A
:104F3000EFC0CFBFE30005FA83278100E3C207FE7D
:104F40008329010183A7490163860700138549006E
:104F5000EFB09F88EFD09FCB83270B00130C050089
:104F60006362F50C8327810017B70100232C875F4C
:104F7000E3E8FBFAB317FA0013F7072163100720E1
:104F800013F7770C6316072A93F70702E38A07F8EB
:104F900013850900EF00504F6FF09FF883A7C700FB
:104FA00003A4C70083AC07009309440013850900DC
:104FB000EFB09F828327440213050400E7800700B7
:104FC0008327C4016386470D8327090003A70700D1
:104FD000E31607FC03A70A0097B6010023A486592D
:104FE00097B6010023A4F65897B7010023A2E7580B
:104FF000EFD0DFF36FF0DFF283A7C70003A4C70091
:1050000003AD0700930C440013850C00EFB0CFFCF8
:105010008327440213050400E78007008327C401A7
:10502000638C470B8327090003A70700E31607FCDF
:1050300003A70A0097B6010023AAF65297B701000A
:1050400023A8E7526FF01FF2EFD0DFBAEFD01FBCFA
:1050500083270B00130C0500E368F5F683A70A000D
:1050600003A504009309000003A60700B385894146
:1050700017B701002328874F13361600EFC0DFAAA9
:10508000EFD0DFEAE31E05E8EFB08FD06FF05FE905
:105090008327840193850900B387FC0063E2FC0841
:1050A00083A7040063860702232A0100232C9101B1
:1050B000232E8100EFF08F9D03A5040093060000CE
:1050C0001306000093054101EFB0DFA6E31E05EED5
:1050D000737004306F0000008327840193850C00F7
:1050E000B307FD006362FD0883A70400638607021F
:1050F000232A0100232CA101232E8100EFF00F9918
:1051000003A5040093060000130600009305410167
:10511000EFB05FA2E31805F0737004306F00000079
:10512000032509002322F40023288400EFB08FE533
:105130006FF09FE9EFD09FDF8327090083A7C700A7
:1051400003A4C700930C440013850C00EFB0CFE814
:105150008327C401638A470583274402130504009B
:10516000E78007006FF0DFDB032509002322F4004E
:1051700023288400EFB00FE16FF0DFEA8327C1003E
:1051800023ACF9006382070AB387870123A2F900E1
:1051900023A83901938549006362FC0803A50A002E
:1051A000EFB04FDE6FF0DFD7832784012328840020
:1051B0003387F9002322E400636AEC04330C3C419A
:1051C000636EFC0283A7040063860702232A0100A2
:1051D000232C3101232E8100EFF04F8B03A5040017
:1051E000930600001306000093054101EFB09F9461
:1051F000E31405F6737004306F00000003A50A0085
:1052000093850C00EFB00FD86FF01FF50325090050
:1052100093850C00EFB00FD76FF01FF40325090042
:10522000EFB04FD66FF0DFCF737004306F00000027
:105230008327C10083A6890123A839013387D700BA
:1052400023A2E9006362EC06B307FC4063EAD706D9
:1052500083A7490213850900E780070083A7C901D6
:10526000E39047CD83A689018327C10003A70400EB
:10527000B387D70063060702232A0100232CF1001D
:10528000232E3101EFF08F8003A504009306000068
:105290001306000093054101EFB0DF89E31205C852
:1052A000737004306F0000006374FC00E372F7FA5F
:1052B0000325090093854900EFB0CFCC6FF05FC69E
:1052C00003A50A0093854900EFB0CFCB6FF05FC50F
:1052D000130101FF232481002326110023229100C2
:1052E0002320210117B4010013040428EFF0CF9903
:1052F0008327040063840704EFF04F9C8327040096
:10530000638A070293080000130800009307000057
:1053100013072000930600001306004097B5010014
:105320009385C50917050000130545B5EFC05F9FBC
:1053300063140506737004306F00000017B9010094
:105340001309894013050900EFB04FBE97B401005F
:105350009384C44013850400EFB04FBD13060000D2
:105360009305C0001305400097B7010023A2272131
:1053700097B7010023AC971EEFB0CFE717B7010036
:105380002324A71E6306050297B5010093858502B5
:10539000EFC04FE66FF05FF68320C1000324810069
:1053A00083244100032901001301010167800000EB
:1053B000737004306F000000638A050A130101FD59
:1053C000232A5101930A05001305C00223248102F8
:1053D0002322910223202103232E3101232C41017A
:1053E00023261102232861012326710113090700D6
:1053F00093890600130A060093840500EF00C0702D
:1054000013040500630C0502EFF00F8897B7010045
:105410009387871583A70700638E0704EFF00F8A31
:105420001305440023205401232C9400232E44010F
:105430002320340323222403EFB04FB113050400CB
:105440008320C10203248102832441020329010233
:105450008329C101032A8101832A4101032B010110
:10546000832BC100130101036780000073700430B7
:105470006F00000097BB0100938B0B2D13850B0071
:10548000EFB0CFAA17BB0100130B4B2D13050B0078
:10549000EFB0CFA9130600009305C000130540002C
:1054A00097B7010023A6770D97B7010023A0670DDA
:1054B000EFB04FD417B701002328A70A630A0500ED
:1054C00097B50100938505EFEFC0CFD26FF01FF5C0
:1054D000737004306F000000630E0506130101FEB7
:1054E000232C8100232E1100232A910017B40100E0
:1054F0001304840783280400130805001305000023
:1055000063800804930407002322B1001387060078
:105510002324C100232601019306500063C0B60472
:10552000EFE0DFD693072000630EF50403250400A7
:10553000930600001306000093054100EFB08FDFD3
:105540008320C1010324810183244101130101024D
:1055500067800000737004306F0000009305410005
:10556000930600001306070013850800EFB05FAE36
:105570008320C1010324810183244101130101021D
:1055800067800000032504009306000013860400D2
:1055900093054100EFB00FDA6FF09FFA6306050044
:1055A0000325050067800000737004306F00000061
:1055B00063160500737004306F000000130101FFD3
:1055C000232611002324810013040500EFE0DFEB04
:1055D000032544013334A000EFE05FEE130504001F
:1055E0008320C100032481001301010167800000B2
:1055F00063160500737004306F000000130101FF93
:10560000232481001304050023261100EFE0DFE7C7
:1056100003240402EFE09FEA8320C1001305040085
:105620000324810013010101678000006316050057
:10563000737004306F000000130101FF2324810008
:1056400023229100138405009304050023261100F2
:10565000EFE09FE323A08402032481008320C100A4
:1056600083244100130101016FE05FE5130101FF95
:105670001305C0012324810023261100EF00C04838
:1056800013040500630805002320050013054500E9
:10569000EFB0CF89130504008320C10003248100EB
:1056A000130101016780000063020502B70700FFD4
:1056B000B3F7F50063860700737004306F000000D5
:1056C000639A0500737004306F000000737004303B
:1056D0006F000000130101FE232C8100232821010B
:1056E000232631012324410123225101232E1100BD
:1056F000232A91009309070013890600930A0600E4
:1057000013840500130A0500EFE05FB86318050075
:1057100063860900737004306F000000EFD08FCDF6
:1057200083240A00B3779400631209046382070498
:1057300063880A009347F4FFB3F797002320FA0029
:10574000EFD0CFFE8320C101032481011385040023
:1057500003290101832441018329C100032A810017
:10576000832A41001301010267800000E302F4FC78
:10577000E38809FCB3355001939585016306090060
:10578000B7070004B3E5F50013860900B3E585000B
:1057900013054A00EFE0CFE1EFD04FF963140500A5
:1057A000EFA01FDFEFE01FD69317650093090500F8
:1057B00063DA0700B70400019384F4FFB3F499009F
:1057C0006FF05FF8EFE05FCC83290A00B377340114
:1057D00063100902638A070063880A009347F4FF95
:1057E000B3F737012320FA00EFE05FCD6FF09FFCA5
:1057F000E31CF4FE6FF05FFE630C0500B70700FFCB
:10580000B3F7F500638A0700737004306F0000007F
:10581000737004306F000000130101FF2324810026
:1058200013040500232611002322910023202101C7
:1058300013890500EFE05FC5832404009345F9FF59
:10584000B3F795002320F400EFE05FC78320C10089
:1058500003248100138504000329010083244100EF
:105860001301010167800000130101FF232481005F
:105870001304050023261100EFA0DFE50324040034
:10588000EFA0DFE48320C10013050400032481009E
:105890001301010167800000630C0500370700FF5A
:1058A000B3F7E500638A0700737004306F000000EF
:1058B000737004306F0000006F30804FB70700FF37
:1058C000B377F60063860700737004306F00000042
:1058D00063160600737004306F000000130101FEB0
:1058E000232C810023282101232631012324410177
:1058F000232E1100232A91001389060093890500A5
:10590000130A050013040600EFE05F98631E050408
:1059100063060900737004306F000000EFD08FAD94
:1059200083240A009385090013050A00B3E4990053
:10593000EFF09FF6B3779400630AF40883240A001B
:10594000EFD0CFDE8320C101032481011385040041
:1059500003290101832441018329C100032A810015
:105960001301010267800000EFD0CFA883240A0052
:105970009385090013050A00B3E43401EFF0DFF169
:10598000B3F7840063848704E30A09FAB7050005C6
:1059900013060900B365B40013054A00EFE04FC1D8
:1059A000EFD0CFD863140500EFA09FBEEFE09FB506
:1059B000931765009304050063D40702B70700013D
:1059C0009387F7FFB3F4F4006FF0DFF783270A0043
:1059D0001344F4FFB3F787002320FA006FF05FF65B
:1059E000EFE09FAA83240A00B377940063988700AE
:1059F0009347F4FFB3F797002320FA00EFE01FACC2
:105A00006FF0DFFB130101FF232481002326110027
:105A10001304050023229100EFD0CF9D832744007B
:105A200063860702032504019304C40063189500EC
:105A30006F0080030325040163089502B705000287
:105A4000EFE04FE183274400E39607FE13050400CF
:105A5000EF008023032481008320C10083244100C0
:105A6000130101016FD08FCC737004306F00000000
:105A7000630C0500370700FFB3F7E500638A0700F2
:105A8000737004306F000000737004306F0000000A
:105A90006F300032630C0500B70700FFB3F7F50065
:105AA000638A0700737004306F0000007370043065
:105AB0006F000000130101FF2324810023229100C5
:105AC000232611001304050093840500EFE0DF9BFB
:105AD0000327040093C7F4FFB377F7002320F400F3
:105AE000032481008320C1008324410013010101AC
:105AF0006FE0DF9C630605000325850167800000D9
:105B00001305000067800000130101FF23248100BA
:105B10002326110013040500EFD0CF8D97B70100A5
:105B2000938747A583A70700639C0704B7970100E5
:105B300017B70100130707C49387C7FF97B6010083
:105B400023A0E6A417B70100232AF7A217B7010084
:105B50002324F7C297B70100938707A217B7010064
:105B6000232AF7C09307100017B70100232C07A0C2
:105B700017B70100232207A017B70100232CF79EB7
:105B800063120402EFD08FBAEF10C06B1304000051
:105B9000130504008320C1000324810013010101C7
:105BA0006780000013058400937735006398070C25
:105BB000B79701001307F5FF9387A7FFE3E4E7FC1E
:105BC00097B601009386C69B83A706006F0040012D
:105BD00003A70700630A07009386070093070700DF
:105BE00003A74700E366A7FE17B701001307C7988E
:105BF000E38AE7F803A70700130600011384870070
:105C000023A0E60003A74700B306A740637ED602A1
:105C10003388A7002322D80023A2A70083254800A9
:105C200097B601009386C6956F0080009306070023
:105C300003A7060003264700E36AB6FE2320E80018
:105C400023A0060103A7470097B701009387479A4F
:105C500083A70700B387E74017B70100232AF79807
:105C6000EFD0CFACE30204F2130504008320C1009F
:105C70000324810013010101678000001375C5FF33
:105C8000130545006FF0DFF263080506130101FFFD
:105C9000232481002326110013040500EFC09FF583
:105CA000930584FF0326C4FF17B701001307478D30
:105CB0006F008000138707008327070083A6470033
:105CC000E3EAC6FE232CF4FE2320B70097B70100B9
:105CD0009387079203A707008327C4FF032481004B
:105CE0008320C100B387E70017B701002322F79094
:105CF000130101016FD08FA36780000097B70100E7
:105D00009387078F03A50700678000006780000066
:105D10003367B50013773700930705006312070454
:105D20009308D6FFB30815011307050093860500F5
:105D30006378150303A806001307470093864600FF
:105D4000232E07FFE36817FF9347F5FFB38717017B
:105D500093F7C7FF93874700B385F500B307F500B6
:105D60003306C50063F4C70C9386450013884700CB
:105D7000B3B6D70033B8050133E7F50093C6160074
:105D80001348180013773700B3E6060113371700DE
:105D90003377D700330EF640938617006308070663
:105DA0001337AE006314070613532E001388050043
:105DB00093860700130700008328080013071700C5
:105DC0001308480023A0160193864600E36667FE89
:105DD0001377CEFFB385E500B387E7006306EE04D3
:105DE00083C60500138717002380D700637EC70290
:105DF00083C6150013872700A380D7006376C702E8
:105E000003C725002381E70067800000B307F64041
:105E1000B387F5009385150003C7F5FF9386160039
:105E2000238FE6FEE398F5FE6780000067800000A0
:105E3000B367C50093F73700B308C5006382070E48
:105E400063761511B307A04093F737001387370027
:105E50009306500093F5F50F130815003383A840FF
:105E60001306F6FF6374D700130750006368E60E4D
:105E70006380070E2300B50013071000638EE70050
:105E8000A300B50013073000130825006396E70050
:105E9000130835002301B5001396850033E6C500CD
:105EA000139705013367E6003303F34093968501AA
:105EB000B366D70013562300B307F500130700009D
:105EC00023A0D7001307170093874700E36AC7FE94
:105ED0001377C3FFB307E8006300E3082380B7002C
:105EE00013871700637C1703A380B700138727006D
:105EF000637617032381B700138737006370170396
:105F0000A381B70013874700637A17012382B70084
:105F10001387570063741701A382B70067800000DE
:105F200093F5F50F13978500B365B7001397050137
:105F30003367B700E37415FF9307050093874700A5
:105F400023AEE7FEE3EC17FF6780000067800000E8
:105F5000130805006FF05FF46780000093070500E9
:105F60006FF0DFF78347050013070500638C070018
:105F70001305150083470500E39C07FE3305E54044
:105F800067800000130500006780000013051500FE
:105F90008347F5FF9385150003C7F5FF6388070066
:105FA000E386E7FE3385E740678000009307000043
:105FB0006FF05FFF930705009385150003C7F5FF9A
:105FC00093871700A38FE7FEE31807FE67800000A2
:105FD00083460500930700026398F6001305150039
:105FE00083460500E38CF6FE938756FD93F7D70FA3
:105FF0006380070493070500930500006388060487
:106000001305000093871700138606FD131725005C
:1060100083C607003305A700131515003305A60036
:10602000E39206FE638405003305A040678000000C
:10603000938536FD8346150093B51500930715002B
:10604000E39006FC130500006FF0DFFD1305000070
:106050006780000083A705002380A70083A70500B1
:106060009387170023A0F5006780000097A6010022
:106070009386865183A7060017370300130787709E
:1060800013861700B307F7002380A70097A5010028
:1060900023ACC54E9307A000630AF50093070004E4
:1060A0006308F6001305000067800000E30C06FE9D
:1060B000370610F0130717008347F7FF2320F6F089
:1060C00083A706009387F7FF97A5010023AEF54A43
:1060D000E39207FE1305000067800000130101EB47
:1060E0002322911423202115232A511323248113C1
:1060F0002326111423248114232E3113232C41131E
:106100002328611323267113232291132320A11323
:10611000232EB11193040500138905002326C10025
:10612000130C5002930A9000834709006388870389
:10613000638C070603A404006F00800063860706D3
:106140002300F40003A4040013091900130414002D
:1061500023A0840083470900E39287FF03461900C8
:106160009308190093860800130D00029309F0FFAD
:10617000130AF0FF13080000130550059307D6FD1E
:1061800093F7F70F13891600636EF53A17A701000E
:10619000130747E793972700B387E70083A7070014
:1061A000B387E700678007008320C11403248114AC
:1061B00083244114032901148329C113032A811361
:1061C000832A4113032B0113832BC112032C811249
:1061D000832C4112032D0112832DC11113010115CE
:1061E00067800000930C80002324010093071000B7
:1061F00063DA071D8327C10003A40400938B770093
:1062000093F68BFF03AB060083A9460093878600B5
:106210002326F10013860C009306000013050B00E3
:1062200093850900EF20C0772328A1009307000081
:1062300063803733930D4101930B100013860C00DC
:106240009306000013050B0093850900EF20003230
:106250009306000013860C00130B050093890500BC
:10626000EF2000748327810023A0AD0093861B00DC
:10627000938D4D0063863701938B06006FF01FFCF2
:10628000E37C9BFF63D24603930704002380A701AE
:1062900003A40400130AFAFF9307140023A0F400D8
:1062A00013840700E3C446FF93962B009307010174
:1062B000B386D7006F008002938777052300F40030
:1062C00003A40400938BFBFF93871B0013041400AB
:1062D00023A084009386C6FFE358F0E483A706005A
:1062E000E3ECFAFC938707036FF05FFD83A70400DC
:1062F000930600030327C1002380D70083A704006F
:1063000093064700930C00011386170023A0C400D6
:1063100013068007A380C70003A404002324010000
:10632000930707001304140023A0840003AB0700A5
:10633000930900002326D1006FF0DFED8327C10011
:1063400083AC0700938B470063880C28635C40256F
:106350009307D002631EFD2083C70C0063880702E9
:1063600063D8092483A60400938C1C00130AFAFF47
:106370002380F60003A404001304140023A0840067
:1063800083C70C00E39E07FC6352400303A4040090
:10639000930700022300F40003A40400130AFAFF89
:1063A0001304140023A08400E3160AFE23267101BF
:1063B0006FF09FD72324010093071000930CA000D7
:1063C000E3CA07E38327C10003A4040093864700C0
:1063D0006FF0DFF503C61600930609006FF01FDAB1
:1063E00083A70400930650022380D70003A404006F
:1063F0001304140023A084006FF01FD3930C00013A
:10640000232401006FF09FDE8327C10003C616001E
:106410009306090083A90700938747002326F1000C
:10642000E35E0AD4138A09009309F0FF6FF01FD5C9
:1064300003C61600130DD002930609006FF01FD497
:106440009347FAFF93D7F74103C61600337AFA0051
:10645000930609006FF09FD203C61600130D0003C8
:10646000930609006FF09FD183C51600930906FDBE
:1064700093060900938705FD13860500E3E2FAFA07
:1064800093972900B38937019386160093991900D1
:10649000B389B90083C50600938909FD938705FD7B
:1064A00013860500E3FEFAFC6FF09FF70327C10097
:1064B00083A7040083260700130747002326E10073
:1064C0002380D70003A404001304140023A0840035
:1064D0006FF09FC59307100063D4070F8327C10097
:1064E0009386770093F686FF938786002326F10034
:1064F00083A9460083A7060063DE090E83A6040075
:106500001306D002B307F0402380C60003A40400A2
:10651000B336F000B30930411304140023A0840003
:10652000138B0700B389D940930CA00023240100EA
:106530006FF05FCE03C6160013081800930609001B
:106540006FF0DFC383A70400138908006FF09FE991
:10655000E3729BCF93071000930B0000930610008B
:10656000E3C447D36FF05FD497AC0100938C8CE504
:106570009385090013850C00EF109037330AAA4069
:106580006352400303A404002300A40103A40400F5
:10659000130AFAFF1304140023A08400E3160AFE72
:1065A000130A000083C70C00E38207E0E3CC09DA9A
:1065B0009389F9FF1307F0FFE396E9DA6FF0DFDC68
:1065C0008327C1009386470083A707002326D100B5
:1065D00093D9F7416FF05FF2635640019307D00201
:1065E000E314FDF897AC0100938CCCDD9307800297
:1065F0006FF01FD7138B0700930CA000232401001A
:1066000003A404006FF01FC1130101EB232E31130B
:10661000B70900409387F9FF2324811423229114A2
:10662000232C4113232A511323261114232021152F
:10663000232861132326711323248113232291130A
:106640002320A113232EB111130A05002324B10026
:1066500017A40100130444F3973A0300938A8A12A3
:1066600097A40100938484AF2326F1009305500280
:106670001305A00013080004B70610F083470A00B2
:10668000638EB7046388070A03270400130A1A00FD
:10669000130617003387EA0097A8010023A6C8EE67
:1066A0002300F7006380A708E31A06FD17370300ED
:1066B0001307470D130717008347F7FF23A0F6F0D2
:1066C000832704009387F7FF17A60100232EF6EA1D
:1066D000E39207FE83470A00E396B7FA83461A005F
:1066E00013051A0013070500930B0002130BF0FFAC
:1066F000130CF0FF13080000930550059308900059
:106700009387D6FD93F7F70F130A170063ECF54450
:1067100093972700B387970083A70700B387970055
:1067200067800700173703001307C705E31406F84F
:106730006FF0DFF48320C1140324811483244114F7
:10674000032901148329C113032A8113832A4113C6
:10675000032B0113832BC112032C8112832C4112B2
:10676000032D0112832DC111130101156780000053
:10677000930C8000130D00009307100063DA0721CB
:10678000832781009387770093F787FF83AD070006
:1067900003AB4700138787002324E10013860C0016
:1067A0009306000013850D0093050B00EF20401F9A
:1067B0002328A10063086D451309410193091000C6
:1067C00013860C009306000013850D0093050B0043
:1067D000EF10D05913860C0093060000930D0500AE
:1067E000138B0500EF20C01B2320A90093891900FB
:1067F00013094900E3166DFDE3F49DFD1306000443
:10680000B70610F063D489038327040013871700A9
:10681000B387FA0097A5010023A8E5D62380770166
:10682000630AC706130CFCFFE3C089FF8327C1007E
:106830001305C10093089000B386F90093962600D3
:1068400093070101B386D7001308A00013030004C7
:10685000370610F0E38CA6E083A70600930500033B
:1068600063F4F8009305700503270400B387B700AD
:10687000930517003387EA0017AE01002326BED028
:106880002300F70063860737638C65329386C6FF63
:106890006FF05FFC173703001307C7EE13071700ED
:1068A0008347F7FF23A0F6F0832704009387F7FFC1
:1068B00097A5010023AAF5CCE39207FE130CFCFF79
:1068C0006FF09FF683270400130600041387170058
:1068D00097A5010023AAE5CAB386FA009305000331
:1068E0002380B6006308C7509387270097A601004E
:1068F00023ACF6C83387EA00930680072300D7004D
:1069000017370300130707E8B70610F06392C702B2
:10691000130717008347F7FF23A0F6F0832704002F
:106920009387F7FF17A601002320F6C6E39207FE20
:1069300083278100930C0001130D0000938747000B
:1069400003278100130B0000832D07002324F1008F
:106950006FF0DFE48327810083AC070013894700D1
:10696000638E0C4C6358802B9307D0026394FB3EDC
:1069700003C70C00930507006314072A6F00002F5C
:1069800093071000930CA000130D0000E3CA07DF6B
:1069900083278100938747006FF09FFA8327810048
:1069A0008346170013070A0003AB070093874700CD
:1069B0002324F100E3560CD4130C0B00130BF0FF4F
:1069C0006FF01FD483461700930BD00213070A0001
:1069D0006FF01FD39347FCFF93D7F741834617000F
:1069E000337CFC0013070A006FF09FD18346170029
:1069F000930B000313070A006FF09FD003461700A4
:106A0000138B06FD13070A00930706FD9306060085
:106A1000E3E2F8FA93172B00B38767011307170017
:106A200093971700B387C70003460700138B07FD32
:106A3000930706FD93060600E3FEF8FC6FF09FF750
:106A400083258100832704001306A00003A7050007
:106A500093861700B387FA0017A501002326D5B245
:106A60002380E700138945006300C73693070004BD
:106A70006384F62A232421016FF05FBF930710007F
:106A800063DE07358327810013877700137787FF3D
:106A9000930787002324F100032B47008327070077
:106AA00063560B3E032704001306000493061700E9
:106AB00097A5010023AAD5AC3387EA009305D0023D
:106AC0002300B700638CC638B307F0403337F000BB
:106AD000330B6041938D0700330BEB40930CA00008
:106AE000130D00006FF09FCB8346170013081800AA
:106AF00013070A006FF0DFC08346170013070A0070
:106B00006FF01FC08327040093060004138717004B
:106B100017A60100232AE6A6B387FA00130650023F
:106B20002380C700E314D7B417370300130787C5C2
:106B3000B70610F0130717008347F7FF23A0F6F0FE
:106B4000832704009387F7FF17A60100232EF6A2E0
:106B5000E39207FE6FF09FB1930C0001130D00004C
:106B60006FF09FC18327040093060004130A0500F9
:106B70001387170017A601002328E6A0B387FA00A1
:106B8000130650022380C700E312D7AE1737030065
:106B9000130747BFB70610F0130717008347F7FF27
:106BA00023A0F6F0832704009387F7FF17A60100C0
:106BB000232CF69CE39207FE130A05006FF01FAB2F
:106BC00017370300130707BC130717008347F7FFA6
:106BD0002320F6F0832704009387F7FF97A5010091
:106BE00023A4F59AE39207FE9386C6FF6FF09FC633
:106BF00017370300130707B9E39805FC9386C6FF10
:106C00006FF05FC5E3FA9DBB930910006FF01FBFE3
:106C1000130C000003C70C0093050700E30C07E406
:106C20009308F0FF1305A00013080004B70610F046
:106C3000635E0B0C8327040013861700B387FA00EA
:106C400017A301002322C3942380E7006382A508D1
:106C50006308060B938C1C0003C70C00130CFCFF8D
:106C600093050700E31607FCE35680E18327040041
:106C70009305000213060004B70610F06F00C00071
:106C8000130CFCFFE3080CDE13871700B387FA0030
:106C90002380B70017A501002328E58E930707007E
:106CA000E310C7FE173703001307C7AD130717001C
:106CB0008347F7FF23A0F6F0832704009387F7FFAD
:106CC00017A501002322F58CE39207FE6FF05FFB0E
:106CD00017370300130707ABE30E06F61307170079
:106CE0008347F7FF23A0F6F0832704009387F7FF7D
:106CF00017A60100232AF688E39207FE6FF09FF59E
:106D000017370300130707A86FF05FFD130BFBFF96
:106D1000E3121BF36FF05FF517370300130787A625
:106D2000B70610F0130717008347F7FF23A0F6F00C
:106D3000832704009387F7FF17A601002326F68414
:106D4000E39207FE232421016FF05F92979C0100DC
:106D5000938C4C6793050B0013850C00EF104039A2
:106D6000330CAC40E35880EB832704001306000487
:106D7000B70610F06F00C000130CFCFFE30A0CE82C
:106D800013871700B387FA002380770197950100D6
:106D900023ACE57E93070700E310C7FE1737030017
:106DA0001307479E130717008347F7FF23A0F6F04A
:106DB000832704009387F7FF9795010023A6F57CAE
:106DC000E39207FE6FF05FFB173703001307879B03
:106DD000E39806F4232421016FF05F898327810063
:106DE0001387470083A707002324E10013DBF74143
:106DF0006FF01FCB173703001307C798B70610F0C3
:106E0000130717008347F7FF23A0F6F0832704003A
:106E10009387F7FF179601002328F676E39207FE83
:106E200093071000179701002320F7769307800738
:106E3000173703002308F7946FF09FAF6356800164
:106E40009307D002E394FBF0979C0100938C8C573E
:106E500013078002930580026FF09FDC97360300D2
:106E600093864692370610F09386160003C7F6FF06
:106E70002320E6F0032704001307F7FF979501008E
:106E800023A4E570E31207FE6FF01FC4938D070083
:106E9000930CA000130D00006FF05F90B70710F087
:106EA00023A0A7F26F000000130101FC13034102AD
:106EB0002322B10293050300232E11002324C102D3
:106EC0002326D1022328E102232AF102232C0103E5
:106ED000232E110323266100EFF00FF38320C1015D
:106EE000130500001301010467800000130101FB7A
:106EF00013038103232481022326A100232CC10232
:106F000013040500130603001305C1002326110214
:106F10002322F104232ED1022320E104232401059E
:106F200023261105232E6100EFF04F9B8327C1001C
:106F3000238007000325C1008320C102330585405B
:106F4000032481021301010567800000B70710F0D8
:106F500083A647F403A607F403A747F4E31AD7FE72
:106F6000B716000093868638B306D60033B6C6003F
:106F7000B305E60023A4D7F423A6B7F46780000086
:106F8000B70710F003A747F403A607F483A647F456
:106F9000E31AD7FEB716000093868638B306D600EC
:106FA00033B6C60023A4D7F4B305E60023A6B7F48E
:106FB0009307000873A0473067800000130101FDAC
:106FC000232481022326110223229102232021035C
:106FD000232E3101232C4101232A51012328610151
:106FE00023267101979701009387875A1794010010
:106FF0001304C45903A70700832704009306470618
:1070000093874706179601002322F658B71700000A
:1070100017960100232ED656938777BB63C8D702F5
:107020008320C10203248102832441020329010237
:107030008329C101032A8101832A4101032B010114
:10704000832BC1001301010367800000B7F7FFFF26
:107050009387C74A3307F7009797010023AAE7529F
:10706000EF000076930710006310F508EF0010336F
:1070700093091000130B4000930B00009304800051
:10708000130AC000930A00001309050063063509BE
:10709000179501001305C535EFF01FE1EF001075DE
:1070A00093040A00630C3509179501001305C536D2
:1070B000EFF09FDF13850400EFF05FDE0324810211
:1070C0008320C10283244102032901028329C101D3
:1070D000032A8101832A4101032B0101832BC10073
:1070E000130101036FB01FB0179501001305052EA2
:1070F000EFF09FDBEF00902A93091000130B600064
:10710000930B20009304A000130AE000930A2000D0
:1071100013090500E31E35F7EF00506DE31625F95E
:1071200063920A0203270400B7270000938777328F
:1071300093040000E3C0E7F86FF09FEE93040B00A8
:107140006FF05FF793840B006FF0DFF61795010087
:107150001305C52E6FF05FD5179501001305852E19
:107160006FF09FD4130101FF23248100232291009B
:1071700023261100B7140000179401001304042DF6
:1071800093878438130000009387F7FFE39C07FE82
:1071900013050400EFF05FD16FF09FFE130101FFB4
:1071A00023261100EF00C058EF00900E8320C1008D
:1071B000130101016F005056130101FF2326110036
:1071C0002324810023229100EF00805F93071000A9
:1071D000631EF5049304400013040000EF00101C2C
:1071E00093071000630AF500179501001305452069
:1071F000EFF09FCB13840400EF00505F9307100063
:10720000630AF5001795010013050521EFF0DFC9AA
:1072100013648400130504008320C100032481004B
:1072200083244100130101016780000017950100CC
:107230001305C519EFF05FC7930460001304200025
:107240006FF0DFF9737004306F000000678000009A
:10725000737004306F000000130101FD23229102BE
:1072600023202103232E3101232C4101232A510104
:10727000232861012326110223248102179A010089
:10728000130A0A33179B0100130BCB3193045005EB
:10729000130910009309E00A930AE00B130500009C
:1072A000EFC0CFFDEFB09F961304050003250A0041
:1072B000930600001306F00A9305C100232601007F
:1072C0009797010023AC972CEF90DF8663060500AB
:1072D0009797010023A6272DEFB05F9333058540D4
:1072E00063F4A90063F6AA009797010023AA272B4D
:1072F000130500009797010023A2972AEFC00FF80B
:10730000EFB0DF901304050003250A009306000088
:107310001306F00A9305C1009797010023A0972850
:10732000EFA0CF80630605009797010023AA2727C7
:10733000EFB0DF8D3305854063F4A90063F6AA0042
:107340009797010023AE27259797010023A897243C
:1073500083270B0093871700179701002324F72436
:107360006FF0DFF3130101FC232A9102232821038C
:1073700023263103232441032322510323206103C5
:10738000232E7101232C8101232A9101232E110226
:10739000232C81022328A101179A0100130A4A21F4
:1073A000179901001309891F979B0100938B0B20EC
:1073B000979C0100938C4C1F130CA000130B100022
:1073C000930A400093091000930450052324010000
:1073D000130600003314CC00EFB05F83130D0500DB
:1073E00003250A0093060000130604009305C1005C
:1073F000EF90DFF3630605009797010023A2371B88
:10740000EFB0DF803305A5419307F4006376850074
:10741000179701002326371963FEA72C0326810046
:107420009797010023AE3717130616002324C100D7
:10743000E3D2CAFA2324010003250A0093060000C0
:107440001306000093058100EF90CFEE6308652DD1
:107450009797010023A6371583278100938717008C
:107460002324F100E3DAFAFC2324010013060000D0
:107470003314CC00EFB08FF9130D050003250A007B
:10748000930600001306040093058100EF908FEA35
:10749000630605009797010023A43711EFB00FF79B
:1074A0003305A5419307F400637685001797010023
:1074B0002328370F63F6A722032681009797010040
:1074C00023A0370F130616002324C100E3D2CAFA03
:1074D00003A50B009797010023A2070CEFB04F9B69
:1074E00083270900638A970013054001EFB05FCF3F
:1074F00083270900E39A97FE13054001EFB05FCEA2
:107500009797010023AC07082324010003250A00F4
:1075100093060000130600009305C100EF901FE1E1
:1075200093060000130600009305810063066501C1
:107530009797010023A6370703250A00EF908FDFF6
:1075400093054000630665019797010023AA37055C
:107550008327090003A50B00639697009797010006
:1075600023A03705EFA09FF883270900930510009B
:1075700003A50B00639697009797010023A237039A
:10758000EFA0DFF683278100938717002324F10003
:10759000E3DEFAF68327090013054001638A9700AA
:1075A000EFB01FC48327090013054001E39A97FE3B
:1075B000EFB01FC39797010023A207FE2324010009
:1075C00003250A0093060000130600009305C1007E
:1075D000EF90DFD5630A65139797010023A237FD6B
:1075E00083278100938717002324F100E3DAFAFC54
:1075F00003A50B00EFB0CF8983270900638A9700AA
:1076000013054001EFB0DFBD83270900E39A97FE21
:1076100013054001EFB0DFBC9797010023A007F8E6
:107620002324010003250A0093060000130600002E
:1076300093058100EF900FD0930600001306000021
:107640009305C100630665019797010023AA37F5EA
:1076500003250A00EF909FCD930540006306650166
:107660009797010023AE37F38327090003A50B008A
:10767000639697009797010023A437F3EFA01FE7C5
:10768000832709009305100003A50B00639697005C
:107690009797010023A637F1EFA05FE583278100CC
:1076A000938717002324F100E3DEFAF6832709000D
:1076B00013054001638A9700EFB09FB2832709004A
:1076C00013054001E39A97FEEFB09FB183A70C002A
:1076D00093871700179701002328F7EC6FF01FCF4F
:1076E00003268100130616002324C100E3D2CAD862
:1076F0006FF01FDE03268100130616002324C1004D
:10770000E3DACACC6FF01FD3832781009387170079
:107710002324F100E3D6FAEA6FF09FED832781007E
:10772000938717002324F100E3D8FAD06FF0DFD35A
:10773000130101FF130600009305400013055000DC
:1077400023261100EF900FAB97950100938545D14B
:107750009797010023AEA7E4EFA0CFA993080000FC
:107760001308000093070000130720009306000091
:1077700013060040979501009385C5CF17050000BB
:10778000130585BEEFA0CFD98320C1009308000068
:107790001308000097970100938747E11307100033
:1077A000930600001306004097950100938505CDD0
:1077B00017050000130585AA130101016FA04FD61C
:1077C00017970100130747DE97960100938686DD21
:1077D00017960100130606DC832707000326060020
:1077E00083A5060017950100130505DB0328050096
:1077F000130500006386C500B38707413335F000E9
:10780000979701009387C7D983A7070083A606002F
:10781000032707009387F7FFB337F000B307F04063
:10782000179601002328D6D63375F50097960100E8
:1078300023A4E6D667800000130101FE232C8100FB
:10784000232E1100232A9100232821012326310110
:1078500023244101032745009307A00A13040500D0
:10786000832405006306F718930600001306000042
:107870009305000013850400EF905FAB93071000A1
:107880006316F5009797010023AAA7D213091000E9
:1078900093091000032A0400930600001306000059
:1078A0009305000013050A00EF905FA86306250FFB
:1078B0009304800C9306000013060000930500005B
:1078C00013050A00EF900FA7832784006308251192
:1078D0009387170017970100232237CF9384F4FF73
:1078E0002324F400E39804FC930600001306000030
:1078F0009305000013050A00EF90CFA3631625013E
:107900009797010023AC27CB032A040093060000BD
:10791000130600009305000013050A00EF908FA1E5
:10792000630225099304800C9306000013060000EF
:107930009305000013050A00EF905F9F83278400E2
:10794000630825079387170017970100232837C777
:107950009384F4FF2324F400E39804FC93060000CE
:10796000130600009305000013050A00EF901F9C0A
:10797000E31225F3032A0400930600001306000017
:107980009305000013050A009797010023A827C359
:10799000EF90DF99E31E25F19797010023A027C3FD
:1079A0006FF01FF19797010023AA27C16FF09FF78F
:1079B000938717009384F4FF2324F400E39604F6DE
:1079C00093060000130600009305000013050A004B
:1079D000EF90DF95E31025ED6FF0DFF99387170047
:1079E0009384F4FF2324F400E39604EC6FF0DFEFBC
:1079F00093060000130600009305000013850400A1
:107A0000EF904F93930710006316F50097970100CE
:107A100023A6A7BA1309800C93091000930600004F
:107A2000130600009305000013850400EF901F90DB
:107A30008327840063043505938717001797010097
:107A4000232E37B71309F9FF2324F400E31809FCA8
:107A50001385040093060000130600009305000040
:107A6000EF90DF8C9307100083240400E31EF5DE03
:107A70009797010023A4A7B46FF01FDF9387170027
:107A80001309F9FF2324F400E31A09F86FF05FFCEF
:107A9000130101FF9305800C1305800C23261100B0
:107AA00023248100EF90CF839727030023ACA7D036
:107AB0009307A00A172703002328F7D09305000097
:107AC0001305800C9727030023A207D0EF904F8166
:107AD0009727030023AEA7CE9727030023AC07CE3A
:107AE00017240300130404CE9727030023A607CE10
:107AF00003250400979501009385C598EF909FEFAB
:107B00000325C400979501009385C598EF909FEEDB
:107B10008327040063880706930800001308000009
:107B2000930700001307000097260300938686C979
:107B300013060040979501009385C5961705000030
:107B40001305C5CFEFA0CF9D032481008320C10082
:107B500093080000130800009307000013070000BB
:107B6000972603009386C6C613060040979501002A
:107B70009385C59317050000130545CC130101013A
:107B80006FA00F9A8327C400E39807F88320C100F1
:107B90000324810013010101678000001797010091
:107BA0001307C7A10326070097270300938787C100
:107BB00017970100130747A00327070083A6870034
:107BC00013050000638AE60003A78700133516003B
:107BD0009796010023A2E69E179701001307879D41
:107BE00083A6470103270700638AE60083A74701AE
:107BF000179701002320F79C678000001305000001
:107C000067800000130101FD2324810223229102D9
:107C100023202103232E3101232C4101232A51014A
:107C200023286101232671012324810123261102C7
:107C3000979401009384849B9799010093894999B3
:107C4000179A0100130A8A98979A0100938A4A9911
:107C5000979B0100938B0B99179C0100130C8C9739
:107C60001304100013093000130B200003A50400B7
:107C700093050000EF909F9BE31A85FE03A5090082
:107C8000EFA04FEA6316250D03250A00EFA08FE948
:107C9000631C250B83A70A00638887009797010060
:107CA00023A487946FF09FFC83A70B00E39887FEC3
:107CB00083270C0003250A009387170017970100FC
:107CC000232AF790EFA0DF9C03A50900EFA05F9C9B
:107CD00083A70A00638C870483A70B00638887044B
:107CE00013050000EFA08FF3631C650503A50900D1
:107CF000EFA04FE36316650703250A00EFA08FE2AC
:107D0000631C650503A50400EF90CFAC63068500F6
:107D10009797010023AA878C13050000EFA00FF0AE
:107D2000E30605F4737004306F00000013050000D3
:107D30009797010023AA878AEFA04FEEE30865FB1F
:107D4000737004306F000000737004306F00000027
:107D5000737004306F000000737004306F00000017
:107D6000737004306F000000130101FE232C8100AA
:107D7000232A9100232821012326310123244101B4
:107D8000232E11001799010013094986179A010043
:107D9000130A4A85979401009384048497990100FB
:107DA0009389C983130410006F0040039797010063
:107DB00023AC878283A7040003A7090093871700D9
:107DC0006386E7009797010023A0878283A70400BA
:107DD00093871700179701002320F78003250900D8
:107DE0009305E0FFEF909F84E31285FC83270A0050
:107DF000E39E87FA03250900EF90CF9D6306850077
:107E00009787010023A2877E130500009787010052
:107E100023A8877CEFB09FC69787010023A2077C29
:107E20006FF05FF9130101FE23282101178901007A
:107E30001309C97B03250900232C81002326310166
:107E4000232E1100232A91001304100097890100AA
:107E50009389C978EF900F986300850A9304A00076
:107E60000325090093058000EF904FFC630C850803
:107E70009384F4FF130540019787010023A68776BA
:107E8000EFB00FB6E39E04FC9304A000130540017D
:107E9000EFB00FB5032509009384F4FFEF908F93A3
:107EA000630685009787010023A08774E39004FE92
:107EB00003250900EF900F92631685009787010054
:107EC00023A4877283A70900130500009387170076
:107ED000178701002324F7709787010023A4877078
:107EE000EFB0DFB9032509009787010023AC076EC7
:107EF000EF904F8EE31485F69787010023A6876ED7
:107F00006FF0DFF59384F4FF13054001EFB04FAD40
:107F1000E39804F46FF05FF7130101FF13054000CD
:107F200023261100EF900F829785010093858558D5
:107F30009787010023ACA76AEF90DFAB978701001A
:107F40009387C76A83A70700638C0708930800001C
:107F500013080000978701009387876713072000A5
:107F60009306000013060040978501009385855510
:107F700017050000130545EBEF909FDA930800000A
:107F800013080000978701009387476413071000C8
:107F90009306000013060040978501009385055362
:107FA00017050000130585DCEF909FD78320C100E3
:107FB0009308000013080000930700001307000057
:107FC00093060000130600409785010093858550B5
:107FD00017050000130545C3130101016F905FD41D
:107FE0008320C10013010101678000009787010011
:107FF0009387C75E978601009386065D03A70700F7
:1080000083A60600638CE60683A707009786010017
:108010009386465B83A60600178701002326F75A3E
:10802000978701009387475B03A70700638CE606E9
:1080300083A70700978601009386865883A60600CB
:10804000178701002320F7589787010093878758E7
:1080500003A70700638CE60683A7070017870100C4
:108060002320F756978701009387075803A5070039
:108070001305F5FF3335A00067800000930710005B
:10808000178701002322F7569786010093868653AF
:10809000978701009387475403A7070083A606002C
:1080A000E398E6F89307100017870100232EF75294
:1080B000978601009386C650978701009387875162
:1080C00003A7070083A60600E398E6F893071000CD
:1080D00017870100232AF750978701009387C7501D
:1080E00003A507001305F5FF3335A00067800000E6
:1080F000B305B500930705006386B70003C7070003
:10810000631607003385A740678000009387170038
:108110006FF09FFE9308000063DC05003305A0406C
:10812000B337A000B305B040B385F5409308F0FF26
:1081300063DA06003306C040B337C000B306D04050
:10814000B386F64013080600138306009307050064
:108150001387050063980624978601009386861589
:1081600063F8C50E370E0100637AC60D130EF00FCB
:108170006374CE0013038000335E6600B386C601CD
:1081800003CE0600330E6E00130300023303C34117
:10819000630C0300B3956500335EC50133186600B8
:1081A0003367BE00B3176500135E0801B355C703FC
:1081B000131508011355050193D607013376C7033C
:1081C000B305B50213160601B366D60063FAB6000E
:1081D000B386060163E6060163F4B600B3860601C2
:1081E000B386B64033F7C6039397070193D70701C9
:1081F000B3D6C603B306D50213150701B367F5005E
:1082000063FAD700B387070163E6070163F4D70079
:10821000B3870701B387D74033D5670093050000C4
:10822000638C0800B307A0403337F000B305B040BB
:1082300013850700B385E54067800000370E000115
:1082400013030001E36AC6F3130380016FF0DFF24A
:108250006316060013081000335868023707010040
:108260006372E80A1307F00F6374070113038000B9
:1082700033576800B386E60003C60600330666007F
:10828000130300023303C34063180308B385054199
:1082900093560801131508011355050113D607015C
:1082A00033F7D502B3D5D502131707013367C700DB
:1082B000B305B502637AB7003307070163660701A8
:1082C0006374B70033070701B305B74033F7D5022E
:1082D0009397070193D70701B3D5D502B305B5022C
:1082E00013150701B367F50063FAB700B3870701F9
:1082F00063E6070163F4B700B3870701B387B740AC
:108300006FF09FF13707000113030001E362E8F605
:10831000130380016FF0DFF53318680033DEC5000A
:10832000935E08013356C500B31765003355DE036D
:10833000B39565003366B6009315080193D5050122
:10834000935606013377DE033385A5021317070121
:108350003367D700637AA700330707016366070115
:108360006374A70033070701B306A74033F7D603AA
:108370001316060113560601B3D6D60313170701C9
:10838000B386D502B365C70063FAD500B38505018E
:1083900063E6050163F4D500B3850501B385D540D7
:1083A0006FF01FEFE3EED5E63708010063FC06052A
:1083B000930EF00F33B8DE001318380033DE0601D9
:1083C00017830100130303EF3303C301834E03003C
:1083D000130E0002B38E0E01330EDE41631E0E0239
:1083E00063E4B600636AC500B307C540B385D540F2
:1083F0003335F5003387A540138507009305070043
:108400006FF01FE23703000113080001E3E866FA8A
:10841000130880016FF09FFA3357D601B396C60157
:10842000B366D700B357D50133D7D501B395C5018E
:10843000B3E7B70093D506013373B702139F060164
:10844000135F0F0113D807013316C6013315C50199
:108450003357B7021313030133680301B30FEF025D
:1084600013030700637EF8013308D8001303F7FFF6
:108470006368D8006376F8011303E7FF3308D80078
:108480003308F841B37FB8023358B802939F0F0105
:10849000B3050F03139F0701135F0F0133EFEF01C4
:1084A00013070800637EBF00330FDF001307F8FFD8
:1084B0006368DF006376BF001307E8FF330FDF0058
:1084C00013130301B70F01003363E3009387FFFF2A
:1084D00013580601330FBF40B375F3001353030164
:1084E000B377F6003387F502B307F302B3850503CC
:1084F00033030303B385F500135807013308B800AD
:108500006374F8003303F301B70701009387F7FFA3
:10851000935508013378F800131808013377F700F2
:10852000B38565003307E8006366BF00631EBF00C4
:10853000637CE5003306C7403337C700B385D540B9
:10854000B385E540130706003307E5403335E50002
:10855000B305BF40B385A540B397D5013357C701D5
:1085600033E5E700B3D5C5016FF09FCB93870500D6
:1085700013080600138706001303050063960628F8
:1085800097880100938808D363F6C50E370701006A
:108590006378E60C1307F00F3337C7001317370063
:1085A000B356E600B388D80083C608003387E600D8
:1085B00093060002B386E640638C0600B397D700AB
:1085C0003357E5003318D600B365F7003313D500F1
:1085D00013550801B3D7A502131608011356060157
:1085E0009356030133F7A502B305F60213170701EB
:1085F000B366D7001387070063FEB600B386060193
:108600001387F7FF63E8060163F6B6001387E7FFF9
:10861000B3860601B386B640B3F7A602131303016F
:1086200013530301B3D6A6029397070133E3670000
:10863000B305D60213850600637CB30033036800DC
:108640001385F6FF636603016374B3001385E6FFC9
:10865000131707013367A700930500006F00400E52
:10866000B706000113070001E36CD6F2130780017F
:108670006FF01FF3631606009306100033D8C6028E
:10868000B70601006372D80C9306F00F63F406017D
:1086900013078000B356E800B388D80083C60800EB
:1086A000B386E600130700023307D7406318070AB2
:1086B000B38707419305100013560801931808016A
:1086C00093D808019356030133F7C702B3D7C70203
:1086D00013170701B366D7003385F8021387070025
:1086E00063FEA600B38606011387F7FF63E8060161
:1086F00063F6A6001387E7FFB3860601B386A6409C
:10870000B3F7C6021313030113530301B3D6C60212
:108710009397070133E36700B388D80213850600F7
:10872000637C1301330368001385F6FF636603015E
:10873000637413011385E6FF131707013367A7005E
:108740001305070067800000B7060001130700014A
:10875000E362D8F4130780016FF0DFF33318E80009
:10876000B3D5D7003313E500B356D5001355080130
:10877000B397E70033F7A502B3E8F60093170801B3
:1087800093D7070113D60801B3D5A5021317070124
:108790003367C700B386B70213860500637ED70030
:1087A000330707011386F5FF636807016376D70077
:1087B0001386E5FF33070701B306D74033F7A60258
:1087C0009398080193D80801B3D6A602131707019E
:1087D000B385D702B36717011387060063FEB7009E
:1087E000B38707011387F6FF63E8070163F6B70055
:1087F0001387E6FFB3870701B387B74093150601D8
:10880000B3E5E5006FF05FEB63E6D51837070100CD
:1088100063F4E6041308F00F3337D800131737005A
:1088200033D8E600978501009385C5A8B385050177
:1088300003C80500930500023308E800B38505412D
:108840006396050213071000E3ECF6EE3335C5001E
:10885000134715006FF0DFEEB705000113070001A5
:10886000E3E0B6FC130780016FF09FFB335706016E
:10887000B396B600B366D70093DE060133D707017F
:10888000B378D703B397B700335805013363F800C3
:108890009397060193D70701135803013316B600C7
:1088A0003357D7039398080133E80801338FE70261
:1088B000130E0700637EE8013308D800130EF7FF9C
:1088C0006368D8006376E801130EE7FF3308D80029
:1088D0003308E841B378D8033358D8039398080194
:1088E000B38E07039317030193D70701B3E7F8008B
:1088F0001307080063FED701B387D7001307F8FFFB
:1089000063E8D70063F6D7011307E8FFB387D70002
:10891000131E0E01B387D741B70E01003367EE0077
:108920001388FEFF3373070193580701337806015C
:1089300013560601330E03033388080393560E01C2
:108940003303C30233030301B3866600B388C8024E
:1089500063F40601B388D80113D60601B3081601E3
:1089600063E61703E39A17CFB70701009387F7FF72
:10897000B3F6F60093960601337EFE003315B5007C
:10898000B386C60193050000E37CD5DA1307F7FF31
:108990006FF09FCC93050000130700006FF05FDAC3
:1089A0009308060013870600930705001388050047
:1089B000639C0622978601009386C68F63FCC50CD4
:1089C00037030100637E660A1303F00F6374C3006C
:1089D000130780003353E600B386660003CE06001B
:1089E00013030002330EEE003303C341630C030094
:1089F000B3956500335EC501B31866003368BE00E9
:108A0000B317650013D608013377C8021395080120
:108A10001355050193D607013358C80213170701F0
:108A2000B366D7003308050363FA0601B38616015F
:108A300063E6160163F40601B3861601B3860641A8
:108A400033F7C6029397070193D70701B3D6C6023F
:108A5000B306D50213150701B367F50063FAD70013
:108A6000B387170163E6170163F4D700B3871701D3
:108A7000B387D74033D567009305000067800000B7
:108A80003703000113070001E36666F41307800152
:108A90006FF05FF46316060013061000B358160358
:108AA0003706010063F2C80A1306F00F637416015B
:108AB0001307800033D6E800B386C60003CE060055
:108AC00013030002330EEE003303C341631803089F
:108AD000B385154113D708011395080113550501F6
:108AE00013D60701B3F6E502B3D5E5029396060166
:108AF000B3E6C600B305B50263FAB600B386160145
:108B000063E6160163F4B600B3861601B385B6407A
:108B1000B3F6E5029397070193D70701B3D5E502B2
:108B2000B305B50213950601B367F50063FAB70004
:108B3000B387170163E6170163F4B700B387170122
:108B4000B387B7406FF01FF337060001130700012A
:108B5000E3E2C8F6130780016FF0DFF5B398680011
:108B600033D7C501B3176500335EC50113D50801BE
:108B7000B376A702B3956500336EBE0093950801E6
:108B800093D5050113560E013357A702939606019C
:108B9000B3E6C6003387E50263FAE600B386160142
:108BA00063E6160163F4E600B38616013386E640F9
:108BB000B376A602131E0E01135E0E013356A602F3
:108BC000939606013386C502B3E5C60163FAC50074
:108BD000B385150163E6150163F4C500B38515017E
:108BE000B385C5406FF01FEFE3EAD5E83707010012
:108BF00063FCE604930EF00F33B7DE001317370063
:108C000033D3E600977801009388C86AB388680078
:108C100083CE0800130E0002B38EEE00330EDE4149
:108C2000631E0E0263E4B600636AC500B307C54065
:108C3000B385D5403335F5003388A540138507004B
:108C4000930508006FF09FE3B708000113070001C8
:108C5000E3E816FB130780016FF09FFA3357D60144
:108C6000B396C601B366D700B357D50133D7D50144
:108C7000B395C501B3E7B70093D506013373B702C7
:108C8000139F0601135F0F0193D807013316C60126
:108C90003315C5013357B70213130301B36813012A
:108CA0003308EF021303070063FE0801B388D800FE
:108CB0001303F7FF63E8D80063F608011303E7FF27
:108CC000B388D800B3880841B3FFB802B3D8B8025C
:108CD000939F0F01B3051F03139F0701135F0F013C
:108CE00033EFEF0113870800637EBF00330FDF000F
:108CF0001387F8FF6368DF006376BF001387E8FF20
:108D0000330FDF0013130301B70801003363E300DF
:108D10009387F8FF13580601330FBF40B375F30074
:108D200013530301B377F6003387F502B307F30259
:108D3000B385050333030303B385F5001358070117
:108D40003308B8006374F80033031301B707010058
:108D50009387F7FF935508013378F800131808013B
:108D60003377F700B38565003307E8006366BF001B
:108D7000631EBF00637CE5003306C7403337C7007E
:108D8000B385D540B385E540130706003307E540BA
:108D90003335E500B305BF40B385A540B397D50192
:108DA0003357C70133E5E700B3D5C5016FF01FCDD9
:108DB000130101FE232C8100232A910013040500D6
:108DC0009384050023282101232631012324410116
:108DD00023225101232E1100EF90DFE183270400AD
:108DE00003290401B7090001B3E59700930AC40001
:108DF0002320B400930400009389F9FF370A00028E
:108E00000327040063822A050326090013050900CD
:108E1000B3654701B37636019317560033F7E60082
:108E20000329490063C60700631607006FF05FFD62
:108E3000E398E6FC9317760063D40700B3E4D4000C
:108E4000EFB04FA16FF0DFFB93C4F4FFB3F4E40085
:108E500023209400EFA08F8D032504008320C101FF
:108E60000324810183244101032901018329C100D5
:108E7000032A8100832A4100130101026780000058
:108E8000130101FF2326110023248100EFE05F8AF4
:108E9000EFE01FC0EFF04F8817E7FFFF13074712FF
:108EA0009306000013061000930540061775010095
:108EB0001305455AEFC04FD06302050213040500A5
:108EC000EF90DFD41306050013070000930600009F
:108ED0009305100013050400EFC00FE0EF901F9EF4
:108EE0008320C10003248100130500001301010148
:048EF0006780000097
:02000004800278
:10000000D463FEFF4465FEFFE063FEFF4465FEFF30
:100010004465FEFF4465FEFF4465FEFF0864FEFF85
:100020004465FEFF4465FEFF3064FEFF4064FEFF52
:100030004465FEFF5864FEFF6864FEFF6864FEFFCF
:100040006864FEFF6864FEFF6864FEFF6864FEFF8C
:100050006864FEFF6864FEFF6864FEFF4465FEFF9F
:100060004465FEFF4465FEFF4465FEFF4465FEFFF8
:100070004465FEFF4465FEFF4465FEFF4465FEFFE8
:100080004465FEFF4465FEFF4465FEFF4465FEFFD8
:100090004465FEFF4465FEFF4465FEFF4465FEFFC8
:1000A0004465FEFF4465FEFF4465FEFF4465FEFFB8
:1000B0004465FEFF4465FEFF4465FEFF4465FEFFA8
:1000C0004465FEFF4465FEFF4465FEFF4465FEFF98
:1000D0004465FEFF4465FEFF4465FEFF4465FEFF88
:1000E0004465FEFF4465FEFF4465FEFF4465FEFF78
:1000F0004465FEFF4465FEFF4465FEFF4465FEFF68
:10010000AC64FEFFD464FEFF4465FEFF4465FEFF61
:100110004465FEFF4465FEFF4465FEFF4465FEFF47
:100120004465FEFF3465FEFF4465FEFF4465FEFF47
:10013000E461FEFFEC62FEFF4465FEFF4465FEFFE6
:100140003C63FEFF4465FEFFB463FEFF4465FEFFB3
:100150004465FEFFFC63FEFFA069FEFF0C6AFEFF24
:10016000AC69FEFF0C6AFEFF0C6AFEFF0C6AFEFF24
:100170000C6AFEFF4468FEFF0C6AFEFF0C6AFEFF7D
:100180006C68FEFF7C68FEFF0C6AFEFF9468FEFF51
:10019000A468FEFFA468FEFFA468FEFFA468FEFF3B
:1001A000A468FEFFA468FEFFA468FEFFA468FEFF2B
:1001B000A468FEFF0C6AFEFF0C6AFEFF0C6AFEFFDD
:1001C0000C6AFEFF0C6AFEFF0C6AFEFF0C6AFEFF63
:1001D0000C6AFEFF0C6AFEFF0C6AFEFF0C6AFEFF53
:1001E0000C6AFEFF0C6AFEFF0C6AFEFF0C6AFEFF43
:1001F0000C6AFEFF0C6AFEFF0C6AFEFF0C6AFEFF33
:100200000C6AFEFF0C6AFEFF0C6AFEFF0C6AFEFF22
:100210000C6AFEFF0C6AFEFF0C6AFEFF0C6AFEFF12
:100220000C6AFEFF0C6AFEFF0C6AFEFF0C6AFEFF02
:100230000C6AFEFF0C6AFEFF0C6AFEFF0C6AFEFFF2
:100240000C6AFEFF0C6AFEFF0C6AFEFF0C6AFEFFE2
:100250000C6AFEFF0C6AFEFFE868FEFF2469FEFFE1
:100260000C6AFEFF0C6AFEFF0C6AFEFF0C6AFEFFC2
:100270000C6AFEFF0C6AFEFF0C6AFEFF9069FEFF2F
:100280000C6AFEFF0C6AFEFF1866FEFF6C67FEFF3D
:100290000C6AFEFF0C6AFEFFFC67FEFF0C6AFEFFA5
:1002A0002868FEFF0C6AFEFF0C6AFEFF006AFEFF74
:1002B000000102020303030304040404040404040D
:1002C00005050505050505050505050505050505DE
:1002D00006060606060606060606060606060606BE
:1002E00006060606060606060606060606060606AE
:1002F000070707070707070707070707070707078E
:10030000070707070707070707070707070707077D
:10031000070707070707070707070707070707076D
:10032000070707070707070707070707070707075D
:10033000080808080808080808080808080808083D
:10034000080808080808080808080808080808082D
:10035000080808080808080808080808080808081D
:10036000080808080808080808080808080808080D
:1003700008080808080808080808080808080808FD
:1003800008080808080808080808080808080808ED
:1003900008080808080808080808080808080808DD
:1003A00008080808080808080808080808080808CD
:1003B000546D725100000000546D7220537663003A
:1003C000286E756C6C2900004572726F7220696E20
:1003D00020626C6F636B2074696D65207465737443
:1003E000207461736B73200D0A0000004572726FF8
:1003F0007220696E20636F756E74696E6720736515
:100400006D6170686F7265207461736B73200D0A83
:10041000000000004572726F7220696E2072656381
:10042000757273697665206D757465782074617373
:100430006B73200D0A0000006D69616F750A000082
:100440006D69616F75320A0068756E6772790A00AE
:10045000436865636B54696D65720000426C6F633D
:100460006B5F54696D655F517565756500000000CF
:100470004254657374310000425465737432000055
:10048000436F756E74696E675F53656D5F31000011
:10049000436F756E74696E675F53656D5F32000000
:1004A000434E543100000000434E5432000000001F
:1004B0005265637572736976655F4D757465780012
:1004C0005265633100000000526563320000000095
:0804D0005265633300000000D7
:1004D8001000000000000000017A5200017C0101B8
:1004E8001B0D02001000000018000000207CFEFF19
:1004F8005804000000000000100000002C0000005C
:100508006480FEFF340400000000000010000000BA
:10051800400000008484FEFF10040000000000007A
:0805EC00FC8F01000400000077
:040000058000004037
:00000001FF
